 libGLESv2

 Timestamp is 4be8c48b (Tue May 11 11:44:27 2010)

 Preferred load address is 10000000

 Start         Length     Name                   Class
 0001:00000000 00000004H .CRT$XCA                CODE
 0001:00000004 00000004H .CRT$XCZ                CODE
 0001:00000008 00000004H .CRT$XIA                CODE
 0001:0000000c 00000004H .CRT$XIZ                CODE
 0001:00000010 00000004H .CRT$XPA                CODE
 0001:00000014 00000004H .CRT$XPZ                CODE
 0001:00000018 00000004H .CRT$XTA                CODE
 0001:0000001c 00000004H .CRT$XTZ                CODE
 0001:00000020 00007df8H .rdata                  CODE
 0001:00007e18 00000026H .rdata$debug            CODE
 0001:00007e40 0003cf04H .text                   CODE
 0001:00044d44 00000028H .xdata                  CODE
 0001:00044d6c 0000003cH .idata$2                CODE
 0001:00044da8 00000014H .idata$3                CODE
 0001:00044dbc 00000148H .idata$4                CODE
 0001:00044f04 0000015aH .idata$6                CODE
 0001:00045060 00000ec9H .edata                  CODE
 0002:00000000 00000148H .idata$5                DATA
 0002:00000148 0000000cH .data                   DATA
 0002:00000154 00000010H .bss                    DATA
 0003:00000000 00001830H .pdata                  DATA

  Address         Publics by Value              Rva+Base       Lib:Object

 0000:00000000       ___safe_se_handler_count   00000000     <absolute>
 0000:00000000       ___safe_se_handler_table   00000000     <absolute>
 0001:00000000       __xc_a                     10001000     corelib0:crt0init.obj
 0001:00000004       __xc_z                     10001004     corelib0:crt0init.obj
 0001:00000008       __xi_a                     10001008     corelib0:crt0init.obj
 0001:0000000c       __xi_z                     1000100c     corelib0:crt0init.obj
 0001:00000010       __xp_a                     10001010     corelib0:crt0init.obj
 0001:00000014       __xp_z                     10001014     corelib0:crt0init.obj
 0001:00000018       __xt_a                     10001018     corelib0:crt0init.obj
 0001:0000001c       __xt_z                     1000101c     corelib0:crt0init.obj
 0001:0000003c       ??_C@_0BH@FPLDHBDI@GL_IMG_program_binary?5?$AA@ 1000103c     accum.obj
 0001:00000054       ??_C@_0BE@FHJHAHOC@GL_IMG_read_format?5?$AA@ 10001054     accum.obj
 0001:00000068       ??_C@_0CA@LDGOBLLP@GL_IMG_texture_format_BGRA8888?5?$AA@ 10001068     accum.obj
 0001:00000088       ??_C@_0BF@LNBCDGHP@GL_IMG_texture_npot?5?$AA@ 10001088     accum.obj
 0001:000000a0       ??_C@_0BI@CMPKADHK@GL_IMG_texture_stream2?5?$AA@ 100010a0     accum.obj
 0001:000000b8       ??_C@_0CC@OEOIKDCE@GL_IMG_texture_compression_pvrtc@ 100010b8     accum.obj
 0001:000000dc       ??_C@_0BG@EIJOAFHK@GL_IMG_shader_binary?5?$AA@ 100010dc     accum.obj
 0001:000000f4       ??_C@_0CA@LLABOCOD@GL_EXT_texture_format_BGRA8888?5?$AA@ 100010f4     accum.obj
 0001:00000114       ??_C@_0BK@HNCIMGED@GL_EXT_multi_draw_arrays?5?$AA@ 10001114     accum.obj
 0001:00000130       ??_C@_0BN@GFHIMELP@GL_OES_standard_derivatives?5?$AA@ 10001130     accum.obj
 0001:00000150       ??_C@_0BN@IPJAGHEM@GL_OES_packed_depth_stencil?5?$AA@ 10001150     accum.obj
 0001:00000170       ??_C@_0BL@BFGJNMLG@GL_OES_get_program_binary?5?$AA@ 10001170     accum.obj
 0001:0000018c       ??_C@_0BG@DDLEGBKL@GL_OES_depth_texture?5?$AA@ 1000118c     accum.obj
 0001:000001a4       ??_C@_0CA@KKMJMEGI@GL_OES_required_internalformat?5?$AA@ 100011a4     accum.obj
 0001:000001c4       ??_C@_0BC@PAMKEGGC@GL_OES_EGL_image?5?$AA@ 100011c4     accum.obj
 0001:000001d8       ??_C@_0CF@IJGGPEFF@GL_OES_compressed_ETC1_RGB8_text@ 100011d8     accum.obj
 0001:00000200       ??_C@_0CA@BJNHKODC@GL_OES_fragment_precision_high?5?$AA@ 10001200     accum.obj
 0001:00000220       ??_C@_0BC@JDOCIJBK@GL_OES_mapbuffer?5?$AA@ 10001220     accum.obj
 0001:00000234       ??_C@_0BL@EKJGK@GL_OES_element_index_uint?5?$AA@ 10001234     accum.obj
 0001:00000250       ??_C@_0BL@PDLBAGFL@GL_OES_texture_half_float?5?$AA@ 10001250     accum.obj
 0001:0000026c       ??_C@_0BG@PANOOMNC@GL_OES_texture_float?5?$AA@ 1000126c     accum.obj
 0001:00000284       ??_C@_0BK@MAHJLLBG@GL_OES_vertex_half_float?5?$AA@ 10001284     accum.obj
 0001:000002a0       ??_C@_0BA@FPFHBIK@GL_OES_depth24?5?$AA@ 100012a0     accum.obj
 0001:000002b0       ??_C@_0BD@OIKJNOON@GL_OES_rgb8_rgba8?5?$AA@ 100012b0     accum.obj
 0001:00000830       ??_C@_0M@FOBNLFJI@1?44?414?42514?$AA@ 10001830     binshader.obj
 0001:0000125c       sGLES2FunctionTable        1000225c     eglglue.obj
 0001:000012d0       ??_C@_0BD@PEKIFPFH@glProgramBinaryOES?$AA@ 100022d0     eglglue.obj
 0001:000012e4       ??_C@_0BG@GMFJDPBI@glGetProgramBinaryOES?$AA@ 100022e4     eglglue.obj
 0001:000012fc       ??_C@_0BD@PIBFHNP@glTexBindStreamIMG?$AA@ 100022fc     eglglue.obj
 0001:00001310       ??_C@_0BM@MBNDOCOP@glGetTexStreamDeviceNameIMG?$AA@ 10002310     eglglue.obj
 0001:0000132c       ??_C@_0CD@OCNNIBKN@glGetTexStreamDeviceAttributeivI@ 1000232c     eglglue.obj
 0001:00001350       ??_C@_0CH@JLEJGINJ@glEGLImageTargetRenderbufferStor@ 10002350     eglglue.obj
 0001:00001378       ??_C@_0BN@FPPCHDBA@glEGLImageTargetTexture2DOES?$AA@ 10002378     eglglue.obj
 0001:00001398       ??_C@_0BE@MPDFJJLL@glMultiDrawElements?$AA@ 10002398     eglglue.obj
 0001:000013ac       ??_C@_0BC@IBABPJFA@glMultiDrawArrays?$AA@ 100023ac     eglglue.obj
 0001:000013c0       ??_C@_0BH@HANHAAH@glGetBufferPointervOES?$AA@ 100023c0     eglglue.obj
 0001:000013d8       ??_C@_0BB@CEFEJGJJ@glUnmapBufferOES?$AA@ 100023d8     eglglue.obj
 0001:000013ec       ??_C@_0P@MBENIONB@glMapBufferOES?$AA@ 100023ec     eglglue.obj
 0001:00001680       ??_C@_0BH@FNCCEFL@OpenGL?5ES?5GLSL?5ES?51?400?$AA@ 10002680     get.obj
 0001:00001698       ??_C@_0O@GGCHPDLB@OpenGL?5ES?52?40?$AA@ 10002698     get.obj
 0001:000016a8       ??_C@_0BA@HGHHDPMC@PowerVR?5SGX?5540?$AA@ 100026a8     get.obj
 0001:000016b8       ??_C@_0BJ@FGEHHHOH@Imagination?5Technologies?$AA@ 100026b8     get.obj
 0001:00001958       pszRenderer                10002958     get.obj
 0001:000020e8       ??_C@_0L@CDGAGNFA@KickTAMode?$AA@ 100030e8     misc.obj
 0001:000020f4       ??_C@_0BA@FMCJLEC@KickTAThreshold?$AA@ 100030f4     misc.obj
 0001:00002104       ??_C@_0BC@DBFGKKHD@OverloadTexLayout?$AA@ 10003104     misc.obj
 0001:00002118       ??_C@_0M@HPPFGNFE@DumpShaders?$AA@ 10003118     misc.obj
 0001:00002124       ??_C@_0BE@CONEIBKK@OptimisedValidation?$AA@ 10003124     misc.obj
 0001:00002138       ??_C@_0BH@EMEDPOLF@DisableHWTextureUpload?$AA@ 10003138     misc.obj
 0001:00002150       ??_C@_0BE@MLGMBNML@DisableHWNormalBlit?$AA@ 10003150     misc.obj
 0001:00002164       ??_C@_0BA@ELLICOAA@DisableHWMipGen?$AA@ 10003164     misc.obj
 0001:00002174       ??_C@_0P@LPEGOECO@FlushBehaviour?$AA@ 10003174     misc.obj
 0001:00002184       ??_C@_0BE@CJIJABHD@EnableStaticMTECopy?$AA@ 10003184     misc.obj
 0001:00002198       ??_C@_0BG@HOCAEBHA@AdjustShaderPrecision?$AA@ 10003198     misc.obj
 0001:000021b0       ??_C@_0BF@LKOMAPLC@DumpCompilerLogFiles?$AA@ 100031b0     misc.obj
 0001:000021c8       ??_C@_0BI@GMOOJAHB@DefaultVertexBufferSize?$AA@ 100031c8     misc.obj
 0001:000021e0       ??_C@_0BH@EMCDMDFL@DefaultIndexBufferSize?$AA@ 100031e0     misc.obj
 0001:000021f8       ??_C@_0BJ@FDELEOJK@DefaultPDSVertBufferSize?$AA@ 100031f8     misc.obj
 0001:00002214       ??_C@_0BF@GMGALNEL@DefaultVDMBufferSize?$AA@ 10003214     misc.obj
 0001:0000222c       ??_C@_0BP@CNJFMOH@DefaultPregenMTECopyBufferSize?$AA@ 1000322c     misc.obj
 0001:0000224c       ??_C@_0BO@DPALACCM@StrictBinaryVersionComparison?$AA@ 1000324c     misc.obj
 0001:0000226c       ??_C@_0BH@KDGMFCIE@PolygonUnitsMultiplier?$AA@ 1000326c     misc.obj
 0001:00002284       ??_C@_0BI@LGOIAELG@PolygonFactorMultiplier?$AA@ 10003284     misc.obj
 0001:0000229c       ??_C@_0BF@ENDLADNG@ForceExternalZBuffer?$AA@ 1000329c     misc.obj
 0001:000022b4       ??_C@_0BH@NAIKDGLA@ForceNoExternalZBuffer?$AA@ 100032b4     misc.obj
 0001:000022cc       ??_C@_0BE@NCEPNDKE@ExternalZBufferMode?$AA@ 100032cc     misc.obj
 0001:000032dc       ??_C@_03EKEJMIG@gl_?$AA@   100042dc     shader.obj
 0001:000032e0       ??_C@_0BB@KACAJBFL@GLSLInitCompiler?$AA@ 100042e0     shader.obj
 0001:000032f4       ??_C@_0BF@OCCHGDEP@GLSLCompileToUniflex?$AA@ 100042f4     shader.obj
 0001:0000330c       ??_C@_0BP@CHEJOEAG@GLSLFreeCompiledUniflexProgram?$AA@ 1000430c     shader.obj
 0001:0000332c       ??_C@_0BD@BNONJEJD@GLSLDisplayMetrics?$AA@ 1000432c     shader.obj
 0001:00003340       ??_C@_0BF@INAJEAID@GLSLShutDownCompiler?$AA@ 10004340     shader.obj
 0001:00003358       ??_C@_0BK@BLBECGOB@SGXBS_CreateBinaryProgram?$AA@ 10004358     shader.obj
 0001:00003374       ??_C@_0N@DJOJPEFE@glslcompiler?$AA@ 10004374     shader.obj
 0001:00003388       ??_C@_0FD@OPILAJHK@The?5active?5size?5of?5?$CFs?5in?5fragmen@ 10004388     shader.obj
 0001:000033dc       ??_C@_0DA@MIAPNJHC@Not?5enough?5contiguous?5indices?5fo@ 100043dc     shader.obj
 0001:0000340c       ??_C@_0DA@PIGCCPJF@No?5built?9in?5attributes?5in?5GLSL?5E@ 1000440c     shader.obj
 0001:0000343c       ??_C@_0CL@HIPONKBO@In?9built?5attributes?5unsupported?5@ 1000443c     shader.obj
 0001:00003468       ??_C@_0EH@JPIEKDIM@Uniform?5variable?5?$CFs?5type?5does?5no@ 10004468     shader.obj
 0001:000034b0       ??_C@_0FB@PELLCLKL@Varying?5variable?5?$CFs?5is?5used?5in?5f@ 100044b0     shader.obj
 0001:00003508       ??_C@_0FH@CHFHBHFF@Active?5size?5for?5varying?5?$CFs?5in?5fr@ 10004508     shader.obj
 0001:00003560       ??_C@_0FG@PMACLKGG@The?5invariance?5for?5varying?5varia@ 10004560     shader.obj
 0001:000035b8       ??_C@_0FA@KBACDFOA@The?5type?5for?5varying?5variable?5?$CFs@ 100045b8     shader.obj
 0001:00004508       TexFormatABGR8888          10005508     texformat.obj
 0001:00004548       TexFormatARGB8888          10005548     texformat.obj
 0001:00004588       TexFormatARGB1555          10005588     texformat.obj
 0001:000045c8       TexFormatARGB4444          100055c8     texformat.obj
 0001:00004608       TexFormatXBGR8888          10005608     texformat.obj
 0001:00004648       TexFormatRGB565            10005648     texformat.obj
 0001:00004688       TexFormatAlpha             10005688     texformat.obj
 0001:000046c8       TexFormatLuminance         100056c8     texformat.obj
 0001:00004708       TexFormatLuminanceAlpha    10005708     texformat.obj
 0001:00004748       TexFormatPVRTC2RGB         10005748     texformat.obj
 0001:00004788       TexFormatPVRTC4RGB         10005788     texformat.obj
 0001:000047c8       TexFormatPVRTC2RGBA        100057c8     texformat.obj
 0001:00004808       TexFormatPVRTC4RGBA        10005808     texformat.obj
 0001:00004848       TexFormatPVRTCII2RGB       10005848     texformat.obj
 0001:00004888       TexFormatPVRTCII4RGB       10005888     texformat.obj
 0001:000048c8       TexFormatPVRTCII2RGBA      100058c8     texformat.obj
 0001:00004908       TexFormatPVRTCII4RGBA      10005908     texformat.obj
 0001:00004948       TexFormatETC1RGB           10005948     texformat.obj
 0001:00004988       TexFormatRGBAFloat         10005988     texformat.obj
 0001:000049c8       TexFormatRGBFloat          100059c8     texformat.obj
 0001:00004a08       TexFormatFloatAlpha        10005a08     texformat.obj
 0001:00004a48       TexFormatFloatLuminance    10005a48     texformat.obj
 0001:00004a88       TexFormatFloatLuminanceAlpha 10005a88     texformat.obj
 0001:00004ac8       TexFormatRGBAHalfFloat     10005ac8     texformat.obj
 0001:00004b08       TexFormatRGBHalfFloat      10005b08     texformat.obj
 0001:00004b48       TexFormatHalfFloatAlpha    10005b48     texformat.obj
 0001:00004b88       TexFormatHalfFloatLuminance 10005b88     texformat.obj
 0001:00004bc8       TexFormatHalfFloatLuminanceAlpha 10005bc8     texformat.obj
 0001:00004c08       TexFormatUYVY              10005c08     texformat.obj
 0001:00004c48       TexFormatYUYV              10005c48     texformat.obj
 0001:00004c88       TexFormatYUV420            10005c88     texformat.obj
 0001:00004cc8       TexFormatFloatDepth        10005cc8     texformat.obj
 0001:00005f40       CopyData                   10006f40     vertex.obj
 0001:00005fb0       MemCopyData                10006fb0     vertex.obj
 0001:00006020       CopyDataShortAligned       10007020     vertex.obj
 0001:00006090       CopyDataByteAligned        10007090     vertex.obj
 0001:00006600       ??_C@_0BA@ELCMJBIB@BufferDevice?$CFd?6?$AA@ 10007600     texstream.obj
 0001:00007968       ??_C@_0DA@NGNCMLGL@PVRUniPatchCreateContext?3?5Contex@ 10008968     usp:usp.obj
 0001:00007998       ??_C@_0EC@BAJDLOCO@PVRUniPatchSetTextureFormat?3?5Inv@ 10008998     usp:usp.obj
 0001:00007e40       InitAccumUSECodeBlocks     10008e40 f   accum.obj
 0001:00008000       FreeAccumUSECodeBlocks     10009000 f   accum.obj
 0001:000085d8       SetupBGObject              100095d8 f   accum.obj
 0001:000088c4       SendAccumulateObject       100098c4 f   accum.obj
 0001:00009804       SGXBS_CreateSharedShaderState 1000a804 f   binshader.obj
 0001:0000997c       SGXBS_CreateProgramState   1000a97c f   binshader.obj
 0001:00009ad4       CreateBufObjState          1000aad4 f   bufobj.obj
 0001:00009af8       FreeBufObjState            1000aaf8 f   bufobj.obj
 0001:00009c5c       SetupBufObjNameArray       1000ac5c f   bufobj.obj
 0001:00009c6c       glBindBuffer               1000ac6c f   bufobj.obj
 0001:00009dd4       glDeleteBuffers            1000add4 f   bufobj.obj
 0001:00009ea0       glGenBuffers               1000aea0 f   bufobj.obj
 0001:00009ee8       glBufferData               1000aee8 f   bufobj.obj
 0001:0000a094       glBufferSubData            1000b094 f   bufobj.obj
 0001:0000a18c       glMapBufferOES             1000b18c f   bufobj.obj
 0001:0000a258       glUnmapBufferOES           1000b258 f   bufobj.obj
 0001:0000a2e0       InitClearUSECodeBlocks     1000b2e0 f   clear.obj
 0001:0000a424       FreeClearUSECodeBlocks     1000b424 f   clear.obj
 0001:0000ab74       SendClearPrims             1000bb74 f   clear.obj
 0001:0000ad80       glClear                    1000bd80 f   clear.obj
 0001:0000aea8       glClearColor               1000bea8 f   clear.obj
 0001:0000af38       glClearDepthf              1000bf38 f   clear.obj
 0001:0000af64       glClearStencil             1000bf64 f   clear.obj
 0001:0000cd10       glDrawArrays               1000dd10 f   drawvarray.obj
 0001:0000cecc       glDrawElements             1000decc f   drawvarray.obj
 0001:0000e0dc       glMultiDrawArrays          1000f0dc f   drawvarray.obj
 0001:0000e450       glMultiDrawElements        1000f450 f   drawvarray.obj
 0001:0000f668       GetColorAttachmentMemFormat 10010668 f   fbo.obj
 0001:0000f6f0       FlushAttachableIfNeeded    100106f0 f   fbo.obj
 0001:0000f7d0       DestroyFBOAttachableRenderSurface 100107d0 f   fbo.obj
 0001:0000f8d8       SetupRenderBufferNameArray 100108d8 f   fbo.obj
 0001:0000f8e8       SetupFrameBufferObjectNameArray 100108e8 f   fbo.obj
 0001:0000f8f8       CreateFrameBufferState     100108f8 f   fbo.obj
 0001:0000f964       RemoveFrameBufferAttachment 10010964 f   fbo.obj
 0001:0000fa80       ChangeDrawableParams       10010a80 f   fbo.obj
 0001:00010478       GetFrameBufferCompleteness 10011478 f   fbo.obj
 0001:00010544       FBOAttachableHasBeenModified 10011544 f   fbo.obj
 0001:00010578       glIsRenderbuffer           10011578 f   fbo.obj
 0001:000105d4       glBindRenderbuffer         100115d4 f   fbo.obj
 0001:00010718       glDeleteRenderbuffers      10011718 f   fbo.obj
 0001:000107d0       glGenRenderbuffers         100117d0 f   fbo.obj
 0001:00010820       glRenderbufferStorage      10011820 f   fbo.obj
 0001:00010af8       SetupRenderbufferFromEGLImage 10011af8 f   fbo.obj
 0001:00010c00       glGetRenderbufferParameteriv 10011c00 f   fbo.obj
 0001:00010d58       glIsFramebuffer            10011d58 f   fbo.obj
 0001:00010db4       glBindFramebuffer          10011db4 f   fbo.obj
 0001:00010f80       glDeleteFramebuffers       10011f80 f   fbo.obj
 0001:00011044       glGenFramebuffers          10012044 f   fbo.obj
 0001:00011090       glCheckFramebufferStatus   10012090 f   fbo.obj
 0001:000110e8       glFramebufferTexture2D     100120e8 f   fbo.obj
 0001:000112b8       glFramebufferRenderbuffer  100122b8 f   fbo.obj
 0001:00011408       glGetFramebufferAttachmentParameteriv 10012408 f   fbo.obj
 0001:00011580       glGenerateMipmap           10012580 f   fbo.obj
 0001:000116a0       FreeFrameBufferState       100126a0 f   fbo.obj
 0001:00012c1c       glGetAttachedShaders       10013c1c f   get.obj
 0001:00012c94       glGetBooleanv              10013c94 f   get.obj
 0001:00012cbc       glGetFloatv                10013cbc f   get.obj
 0001:00012ce4       glGetIntegerv              10013ce4 f   get.obj
 0001:00012d0c       glGetBufferParameteriv     10013d0c f   get.obj
 0001:00012df8       glGetBufferPointervOES     10013df8 f   get.obj
 0001:00012ea0       glGetError                 10013ea0 f   get.obj
 0001:00012ec4       glGetShaderiv              10013ec4 f   get.obj
 0001:00012fc8       glGetProgramiv             10013fc8 f   get.obj
 0001:0001330c       glGetProgramInfoLog        1001430c f   get.obj
 0001:000133ac       glGetShaderInfoLog         100143ac f   get.obj
 0001:0001344c       glGetShaderSource          1001444c f   get.obj
 0001:000134ec       glGetString                100144ec f   get.obj
 0001:00013764       glGetTexParameteriv        10014764 f   get.obj
 0001:00013794       glGetTexParameterfv        10014794 f   get.obj
 0001:000137d8       glGetUniformfv             100147d8 f   get.obj
 0001:00013870       glGetUniformiv             10014870 f   get.obj
 0001:00013944       glGetAttribLocation        10014944 f   get.obj
 0001:00013a1c       glGetVertexAttribfv        10014a1c f   get.obj
 0001:00013c14       glGetVertexAttribiv        10014c14 f   get.obj
 0001:00013da8       glGetVertexAttribPointerv  10014da8 f   get.obj
 0001:00013e00       glIsEnabled                10014e00 f   get.obj
 0001:00013e24       glIsBuffer                 10014e24 f   get.obj
 0001:00013e80       glIsProgram                10014e80 f   get.obj
 0001:00013ee8       glIsShader                 10014ee8 f   get.obj
 0001:00013f50       glIsTexture                10014f50 f   get.obj
 0001:00013fac       glGetShaderPrecisionFormat 10014fac f   get.obj
 0001:000153ec       MakeTextureMipmapLevels    100163ec f   makemips.obj
 0001:000159e0       Clampf                     100169e0 f   misc.obj
 0001:00015a44       Clampi                     10016a44 f   misc.obj
 0001:00015c70       ColorConvertToHWFormat     10016c70 f   misc.obj
 0001:00015cb4       FloorLog2                  10016cb4 f   misc.obj
 0001:00015cd4       GLES2ConvertFloatToF16     10016cd4 f   misc.obj
 0001:00015dd8       GLES2ConvertFloatToC10     10016dd8 f   misc.obj
 0001:00015ea0       BuildExtensionString       10016ea0 f   misc.obj
 0001:00015f3c       DestroyExtensionString     10016f3c f   misc.obj
 0001:00015f58       GetApplicationHints        10016f58 f   misc.obj
 0001:00016358       SetError                   10017358 f   misc.obj
 0001:00016370       glFinish                   10017370 f   misc.obj
 0001:00016488       glFlush                    10017488 f   misc.obj
 0001:000164c8       glHint                     100174c8 f   misc.obj
 0001:00016544       SetErrorFRM                10017544 f   misc.obj
 0001:00016568       CreateNamesArray           10017568 f   names.obj
 0001:00016608       NamesArrayGenNames         10017608 f   names.obj
 0001:000166d0       NamesArrayMapFunction      100176d0 f   names.obj
 0001:00016744       DestroyNamesArray          10017744 f   names.obj
 0001:000167a0       InsertNamedItem            100177a0 f   names.obj
 0001:00016874       NamedItemAddRef            10017874 f   names.obj
 0001:00016904       NamedItemDelRef            10017904 f   names.obj
 0001:000169dc       NamedItemDelRefByName      100179dc f   names.obj
 0001:00016b38       glPixelStorei              10017b38 f   pixelop.obj
 0001:00016db0       SetupReadPixelsSpanInfo    10017db0 f   pixelop.obj
 0001:00017188       glReadPixels               10018188 f   pixelop.obj
 0001:0001745c       InitScissorUSECodeBlocks   1001845c f   scissor.obj
 0001:000174d4       FreeScissorUSECodeBlocks   100184d4 f   scissor.obj
 0001:00017db0       SendDrawMaskForPrimitive   10018db0 f   scissor.obj
 0001:00017f88       SendDrawMaskForClear       10018f88 f   scissor.obj
 0001:00018050       glScissor                  10019050 f   scissor.obj
 0001:00018128       WaitForTA                  10019128 f   sgxif.obj
 0001:0001863c       PrepareToDraw              1001963c f   sgxif.obj
 0001:00018f0c       ScheduleTA                 10019f0c f   sgxif.obj
 0001:00019088       KickLimit_ScheduleTA       1001a088 f   sgxif.obj
 0001:000190ac       USESecondaryUploadTaskAddRef 1001a0ac f   shader.obj
 0001:000190ec       USESecondaryUploadTaskDelRef 1001a0ec f   shader.obj
 0001:000194e4       GetNamedProgram            1001a4e4 f   shader.obj
 0001:00019548       GetNamedShader             1001a548 f   shader.obj
 0001:000195ac       glAttachShader             1001a5ac f   shader.obj
 0001:00019664       glDetachShader             1001a664 f   shader.obj
 0001:00019738       glBindAttribLocation       1001a738 f   shader.obj
 0001:00019850       glCreateProgram            1001a850 f   shader.obj
 0001:0001991c       glDeleteProgram            1001a91c f   shader.obj
 0001:00019978       glCreateShader             1001a978 f   shader.obj
 0001:00019a60       glDeleteShader             1001aa60 f   shader.obj
 0001:00019ac0       glGetActiveAttrib          1001aac0 f   shader.obj
 0001:00019f1c       DestroyGLSLCompiler        1001af1c f   shader.obj
 0001:00019f78       UniPatchMalloc             1001af78 f   shader.obj
 0001:00019f7c       UniPatchFree               1001af7c f   shader.obj
 0001:00019f80       UniPatchDebugPrint         1001af80 f   shader.obj
 0001:00019f90       DestroyHashedPDSVariant    1001af90 f   shader.obj
 0001:0001b170       glUseProgram               1001c170 f   shader.obj
 0001:0001b18c       glValidateProgram          1001c18c f   shader.obj
 0001:0001b2e8       glReleaseShaderCompiler    1001c2e8 f   shader.obj
 0001:0001b2fc       glShaderSource             1001c2fc f   shader.obj
 0001:0001b440       glGetProgramBinaryOES      1001c440 f   shader.obj
 0001:0001b6fc       FreeProgramState           1001c6fc f   shader.obj
 0001:0001b7a4       DestroyUSEShaderVariant    1001c7a4 f   shader.obj
 0001:0001b874       DestroyUSEShaderVariantGhost 1001c874 f   shader.obj
 0001:0001b9d8       ReclaimUSEShaderVariantMemFRM 1001c9d8 f   shader.obj
 0001:0001b9e0       DestroyUSECodeVariantGhostFRM 1001c9e0 f   shader.obj
 0001:0001ba54       DestroyVertexVariants      1001ca54 f   shader.obj
 0001:0001bc5c       glLinkProgram              1001cc5c f   shader.obj
 0001:0001be00       glCompileShader            1001ce00 f   shader.obj
 0001:0001c0a8       glShaderBinary             1001d0a8 f   shader.obj
 0001:0001c1bc       glProgramBinaryOES         1001d1bc f   shader.obj
 0001:0001c624       SetupProgramNameArray      1001d624 f   shader.obj
 0001:0001c634       CreateProgramState         1001d634 f   shader.obj
 0001:0001c750       SpanPack16                 1001d750 f   spanpack.obj
 0001:0001c798       SpanPack32                 1001d798 f   spanpack.obj
 0001:0001c7e0       SpanPackARGB4444toRGBA4444 1001d7e0 f   spanpack.obj
 0001:0001c814       SpanPackARGB1555toRGBA5551 1001d814 f   spanpack.obj
 0001:0001c848       SpanPackARGB8888toABGR8888 1001d848 f   spanpack.obj
 0001:0001c890       SpanPackARGB8888toXBGR8888 1001d890 f   spanpack.obj
 0001:0001c8d8       SpanPackARGB8888toRGB565   1001d8d8 f   spanpack.obj
 0001:0001c928       SpanPackARGB8888toARGB4444 1001d928 f   spanpack.obj
 0001:0001c980       SpanPackARGB8888toARGB1555 1001d980 f   spanpack.obj
 0001:0001c9d4       SpanPackARGB8888toLuminanceAlpha 1001d9d4 f   spanpack.obj
 0001:0001ca00       SpanPackARGB8888toLuminance 1001da00 f   spanpack.obj
 0001:0001ca2c       SpanPackAXXX8888toAlpha    1001da2c f   spanpack.obj
 0001:0001ca58       SpanPackABGR8888toARGB8888 1001da58 f   spanpack.obj
 0001:0001caa0       SpanPackABGR8888toXBGR8888 1001daa0 f   spanpack.obj
 0001:0001cae8       SpanPackABGR8888toRGB565   1001dae8 f   spanpack.obj
 0001:0001cb38       SpanPackABGR8888toARGB4444 1001db38 f   spanpack.obj
 0001:0001cb90       SpanPackABGR8888toARGB1555 1001db90 f   spanpack.obj
 0001:0001cbe8       SpanPackABGR8888toLuminanceAlpha 1001dbe8 f   spanpack.obj
 0001:0001cc20       SpanPackABGR8888toLuminance 1001dc20 f   spanpack.obj
 0001:0001cc4c       SpanPackARGB4444toABGR8888 1001dc4c f   spanpack.obj
 0001:0001ccb4       SpanPackARGB4444toXBGR8888 1001dcb4 f   spanpack.obj
 0001:0001cd14       SpanPackARGB4444toARGB8888 1001dd14 f   spanpack.obj
 0001:0001cd7c       SpanPackARGB4444toRGB565   1001dd7c f   spanpack.obj
 0001:0001cdf8       SpanPackARGB4444toARGB1555 1001ddf8 f   spanpack.obj
 0001:0001ce7c       SpanPackARGB4444toLuminanceAlpha 1001de7c f   spanpack.obj
 0001:0001cec8       SpanPackARGB4444toLuminance 1001dec8 f   spanpack.obj
 0001:0001cefc       SpanPackARGB4444toAlpha    1001defc f   spanpack.obj
 0001:0001cf30       SpanPackARGB1555toABGR8888 1001df30 f   spanpack.obj
 0001:0001cfa4       SpanPackARGB1555toXBGR8888 1001dfa4 f   spanpack.obj
 0001:0001d010       SpanPackARGB1555toARGB8888 1001e010 f   spanpack.obj
 0001:0001d07c       SpanPackARGB1555toRGB565   1001e07c f   spanpack.obj
 0001:0001d0d8       SpanPackARGB1555toARGB4444 1001e0d8 f   spanpack.obj
 0001:0001d128       SpanPackARGB1555toLuminanceAlpha 1001e128 f   spanpack.obj
 0001:0001d17c       SpanPackARGB1555toLuminance 1001e17c f   spanpack.obj
 0001:0001d1b8       SpanPackARGB1555toAlpha    1001e1b8 f   spanpack.obj
 0001:0001d1f8       SpanPackRGB565toXBGR8888   1001e1f8 f   spanpack.obj
 0001:0001d260       SpanPackRGB565toLuminance  1001e260 f   spanpack.obj
 0001:0001d294       glBlendColor               1001e294 f   state.obj
 0001:0001d344       glBlendEquation            1001e344 f   state.obj
 0001:0001d3c0       glBlendEquationSeparate    1001e3c0 f   state.obj
 0001:0001d65c       glBlendFuncSeparate        1001e65c f   state.obj
 0001:0001d698       glBlendFunc                1001e698 f   state.obj
 0001:0001d6cc       glColorMask                1001e6cc f   state.obj
 0001:0001d744       glCullFace                 1001e744 f   state.obj
 0001:0001d7b4       glDepthFunc                1001e7b4 f   state.obj
 0001:0001d80c       glDepthMask                1001e80c f   state.obj
 0001:0001d85c       ApplyDepthRange            1001e85c f   state.obj
 0001:0001d95c       glDepthRangef              1001e95c f   state.obj
 0001:0001d980       glDisable                  1001e980 f   state.obj
 0001:0001daac       glEnable                   1001eaac f   state.obj
 0001:0001dbd8       glFrontFace                1001ebd8 f   state.obj
 0001:0001dc30       glLineWidth                1001ec30 f   state.obj
 0001:0001dcc4       glPolygonOffset            1001ecc4 f   state.obj
 0001:0001dd38       glSampleCoverage           1001ed38 f   state.obj
 0001:0001df14       glStencilFunc              1001ef14 f   state.obj
 0001:0001df50       glStencilFuncSeparate      1001ef50 f   state.obj
 0001:0001e070       glStencilMask              1001f070 f   state.obj
 0001:0001e0ec       glStencilMaskSeparate      1001f0ec f   state.obj
 0001:0001e2a8       glStencilOp                1001f2a8 f   state.obj
 0001:0001e2e8       glStencilOpSeparate        1001f2e8 f   state.obj
 0001:0001e328       ApplyViewport              1001f328 f   state.obj
 0001:0001e4c8       glViewport                 1001f4c8 f   state.obj
 0001:0001e5d4       HashTableCreate            1001f5d4 f   statehash.obj
 0001:0001e62c       HashTableDestroy           1001f62c f   statehash.obj
 0001:0001e6b0       HashFunc                   1001f6b0 f   statehash.obj
 0001:0001e6e0       HashTableSearch            1001f6e0 f   statehash.obj
 0001:0001e798       HashTableDelete            1001f798 f   statehash.obj
 0001:0001e8c0       HashTableInsert            1001f8c0 f   statehash.obj
 0001:0001e9d4       CopyTextureFloatRGBA       1001f9d4 f   tex.obj
 0001:0001ea64       CopyTextureFloatRGB        1001fa64 f   tex.obj
 0001:0001eae8       CopyTextureFloatLA         1001fae8 f   tex.obj
 0001:0001eb54       CopyTextureHalfFloatRGBA   1001fb54 f   tex.obj
 0001:0001ebd4       CopyTextureHalfFloatRGB    1001fbd4 f   tex.obj
 0001:0001ec4c       CopyTextureBGRA8888toRGBA8888 1001fc4c f   tex.obj
 0001:0001ecc4       CopyTextureBGRA8888to5551  1001fcc4 f   tex.obj
 0001:0001ed50       CopyTextureBGRA8888to4444  1001fd50 f   tex.obj
 0001:0001eed8       CopyTexture32Bits          1001fed8 f   tex.obj
 0001:0001ef2c       CopyTexture16Bits          1001ff2c f   tex.obj
 0001:0001ef80       CopyTexture8Bits           1001ff80 f   tex.obj
 0001:0001efd4       CopyTexture16BitIntTo32BitFloat 1001ffd4 f   tex.obj
 0001:0001f078       CopyTexture32BitIntTo32BitFloat 10020078 f   tex.obj
 0001:0001f11c       CopyTexture5551            1002011c f   tex.obj
 0001:0001f178       CopyTexture4444            10020178 f   tex.obj
 0001:0001f1d4       CopyTexture888X            100201d4 f   tex.obj
 0001:0001f248       CopyTexture888to565        10020248 f   tex.obj
 0001:0001f2cc       CopyTexture565toRGBX8888   100202cc f   tex.obj
 0001:0001f348       CopyTexture5551to4444      10020348 f   tex.obj
 0001:0001f3e8       CopyTexture5551toBGRA8888  100203e8 f   tex.obj
 0001:0001f474       CopyTexture5551toRGBA8888  10020474 f   tex.obj
 0001:0001f500       CopyTexture4444to5551      10020500 f   tex.obj
 0001:0001f59c       CopyTexture4444toRGBA8888  1002059c f   tex.obj
 0001:0001f61c       CopyTextureRGBA8888to5551  1002061c f   tex.obj
 0001:0001f6ac       CopyTextureRGBA8888to4444  100206ac f   tex.obj
 0001:0001f9c0       glTexParameteri            100209c0 f   tex.obj
 0001:0001f9f8       glTexParameterf            100209f8 f   tex.obj
 0001:0001fa54       glTexParameteriv           10020a54 f   tex.obj
 0001:0001fa90       glTexParameterfv           10020a90 f   tex.obj
 0001:0001faec       glActiveTexture            10020aec f   tex.obj
 0001:0001fb30       BindTexture                10020b30 f   tex.obj
 0001:0001fc80       glBindTexture              10020c80 f   tex.obj
 0001:0001fd24       glDeleteTextures           10020d24 f   tex.obj
 0001:0001fe2c       glGenTextures              10020e2c f   tex.obj
 0001:000201ec       glTexImage2D               100211ec f   tex.obj
 0001:0002092c       glTexSubImage2D            1002192c f   tex.obj
 0001:00021478       glCompressedTexImage2D     10022478 f   tex.obj
 0001:0002171c       glCompressedTexSubImage2D  1002271c f   tex.obj
 0001:000218e8       glCopyTexImage2D           100228e8 f   tex.obj
 0001:00021ef8       glCopyTexSubImage2D        10022ef8 f   tex.obj
 0001:00022f28       HardwareSubTextureUpload   10023f28 f   texdata.obj
 0001:000234f8       HardwareCopySubTextureUpload 100244f8 f   texdata.obj
 0001:00023848       HardwareTextureUpload      10024848 f   texdata.obj
 0001:00023b94       ReadBackTiledData          10024b94 f   texdata.obj
 0001:00023cf8       GetMipMapOffset            10024cf8 f   texdata.obj
 0001:00023d24       GetCompressedMipMapOffset  10024d24 f   texdata.obj
 0001:00023d98       GetNPOTMipMapOffset        10024d98 f   texdata.obj
 0001:00023e54       TranslateLevel             10024e54 f   texdata.obj
 0001:000243f4       SetupTwiddleFns            100253f4 f   texdata.obj
 0001:00024444       CopyTextureData            10025444 f   texdata.obj
 0001:0002467c       ReadBackTextureData        1002567c f   texdata.obj
 0001:00024a74       ReclaimTextureMemFRM       10025a74 f   texmgmt.obj
 0001:00024b48       DestroyTextureGhostFRM     10025b48 f   texmgmt.obj
 0001:00024ba0       CreateTextureMemory        10025ba0 f   texmgmt.obj
 0001:00024dec       TexMgrGhostTexture         10025dec f   texmgmt.obj
 0001:00024ed8       TextureRemoveResident      10025ed8 f   texmgmt.obj
 0001:00024ee4       TextureMakeResident        10025ee4 f   texmgmt.obj
 0001:000252b4       IsTextureConsistent        100262b4 f   texmgmt.obj
 0001:00025834       TextureCreateImageLevel    10026834 f   texmgmt.obj
 0001:00025a44       TextureCreateLevel         10026a44 f   texmgmt.obj
 0001:00025b9c       CreateTexture              10026b9c f   texmgmt.obj
 0001:00025ea0       CreateTextureState         10026ea0 f   texmgmt.obj
 0001:00025f38       SetupTexNameArray          10026f38 f   texmgmt.obj
 0001:00025f48       ReleaseTextureManager      10026f48 f   texmgmt.obj
 0001:00025f98       FreeTextureState           10026f98 f   texmgmt.obj
 0001:00026020       SetupTextureState          10027020 f   texmgmt.obj
 0001:00026528       SetupTextureRenderTargetControlWords 10027528 f   texmgmt.obj
 0001:00026790       CreateTextureManager       10027790 f   texmgmt.obj
 0001:00026840       ConvertGLSLtoGLType        10027840 f   uniform.obj
 0001:00026850       SetupBuiltInUniforms       10027850 f   uniform.obj
 0001:00026b38       WriteUSEShaderMemConsts    10027b38 f   uniform.obj
 0001:000275b4       GetUniformData             100285b4 f   uniform.obj
 0001:00027704       FindUniformFromLocation    10028704 f   uniform.obj
 0001:00027758       glGetActiveUniform         10028758 f   uniform.obj
 0001:00027834       glGetUniformLocation       10028834 f   uniform.obj
 0001:0002798c       glUniform1i                1002898c f   uniform.obj
 0001:00027a88       glUniform2i                10028a88 f   uniform.obj
 0001:00027b40       glUniform3i                10028b40 f   uniform.obj
 0001:00027c00       glUniform4i                10028c00 f   uniform.obj
 0001:00027cc8       glUniform1f                10028cc8 f   uniform.obj
 0001:00027d74       glUniform2f                10028d74 f   uniform.obj
 0001:00027e2c       glUniform3f                10028e2c f   uniform.obj
 0001:00027eec       glUniform4f                10028eec f   uniform.obj
 0001:00027fb4       glUniform1iv               10028fb4 f   uniform.obj
 0001:000280d8       glUniform2iv               100290d8 f   uniform.obj
 0001:000281a0       glUniform3iv               100291a0 f   uniform.obj
 0001:00028268       glUniform4iv               10029268 f   uniform.obj
 0001:00028330       glUniform1fv               10029330 f   uniform.obj
 0001:000283d8       glUniform2fv               100293d8 f   uniform.obj
 0001:000284a0       glUniform3fv               100294a0 f   uniform.obj
 0001:00028568       glUniform4fv               10029568 f   uniform.obj
 0001:00028630       glUniformMatrix2fv         10029630 f   uniform.obj
 0001:00028710       glUniformMatrix3fv         10029710 f   uniform.obj
 0001:000287f0       glUniformMatrix4fv         100297f0 f   uniform.obj
 0001:00028b74       GetFBBlendType             10029b74 f   use.obj
 0001:00028cc0       CreateFBBlendUSECode       10029cc0 f   use.obj
 0001:00028e84       CreateColorMaskUSECode     10029e84 f   use.obj
 0001:00028eec       WriteEOTUSSECode           10029eec f   use.obj
 0001:00028ff0       GetStateCopyUSEAddress     10029ff0 f   use.obj
 0001:000290fc       InitSpecialUSECodeBlocks   1002a0fc f   use.obj
 0001:000291b4       FreeSpecialUSECodeBlocks   1002a1b4 f   use.obj
 0001:000299cc       SetupUSEVertexShader       1002a9cc f   use.obj
 0001:00029f9c       SetupUSEFragmentShader     1002af9c f   use.obj
 0001:0002a690       EncodeDmaBurst             1002b690 f   validate.obj
 0001:0002a73c       OutputTerminateState       1002b73c f   validate.obj
 0001:0002a8ec       SetupPixelEventProgram     1002b8ec f   validate.obj
 0001:0002c4e8       PatchPregenMTEStateCopyPrograms 1002d4e8 f   validate.obj
 0001:0002c630       WriteMTEStateCopyPrograms  1002d630 f   validate.obj
 0001:0002c784       SetupStateUpdate           1002d784 f   validate.obj
 0001:0002c888       SetupMTEPregenBuffer       1002d888 f   validate.obj
 0001:0002d134       ValidateState              1002e134 f   validate.obj
 0001:0002d2e0       GLES2EmitState             1002e2e0 f   validate.obj
 0001:0002db24       glEnableVertexAttribArray  1002eb24 f   vertex.obj
 0001:0002db74       glDisableVertexAttribArray 1002eb74 f   vertex.obj
 0001:0002dbc4       glVertexAttrib1f           1002ebc4 f   vertex.obj
 0001:0002dc10       glVertexAttrib2f           1002ec10 f   vertex.obj
 0001:0002dc60       glVertexAttrib3f           1002ec60 f   vertex.obj
 0001:0002dcb0       glVertexAttrib4f           1002ecb0 f   vertex.obj
 0001:0002dd00       glVertexAttrib1fv          1002ed00 f   vertex.obj
 0001:0002dd50       glVertexAttrib2fv          1002ed50 f   vertex.obj
 0001:0002dda4       glVertexAttrib3fv          1002eda4 f   vertex.obj
 0001:0002ddf8       glVertexAttrib4fv          1002edf8 f   vertex.obj
 0001:0002de4c       glVertexAttribPointer      1002ee4c f   vertex.obj
 0001:0002dfec       ReleaseImageFromTexture    1002efec f   eglimage.obj
 0001:0002e158       glEGLImageTargetTexture2DOES 1002f158 f   eglimage.obj
 0001:0002e274       glEGLImageTargetRenderbufferStorageOES 1002f274 f   eglimage.obj
 0001:0002e31c       ReleaseImageFromRenderbuffer 1002f31c f   eglimage.obj
 0001:0002e33c       GLESGetImageSource         1002f33c f   eglimage.obj
 0001:0002e83c       SetupYUVCoefficients       1002f83c f   texstream.obj
 0001:0002eb3c       GetNumStreamDevices        1002fb3c f   texstream.obj
 0001:0002eb70       FreeTexStreamState         1002fb70 f   texstream.obj
 0001:0002ed9c       FindBufferDevice           1002fd9c f   texstream.obj
 0001:0002edd4       AddBufferDevice            1002fdd4 f   texstream.obj
 0001:0002f098       glGetTexStreamDeviceAttributeivIMG 10030098 f   texstream.obj
 0001:0002f194       glTexBindStreamIMG         10030194 f   texstream.obj
 0001:0002f340       glGetTexStreamDeviceNameIMG 10030340 f   texstream.obj
 0001:0002f3b8       OGLES2_GetTLSValue         100303b8 f   wince6_tls.obj
 0001:0002f3e8       OGLES2_SetTLSValue         100303e8 f   wince6_tls.obj
 0001:0002f42c       PDSGeneratePixelEventProgram 1003042c f   pds.obj
 0001:0002f548       PDSPatchVertexShaderProgram 10030548 f   pds.obj
 0001:0002f674       PDSGeneratePixelShaderSAProgram 10030674 f   pds.obj
 0001:0002f91c       PDSGeneratePixelShaderProgram 1003091c f   pds.obj
 0001:0002fb6c       PDSGenerateStateCopyProgram 10030b6c f   pds.obj
 0001:0002fcdc       PDSGenerateVertexShaderProgram 10030cdc f   pds.obj
 0001:000303a8       PDSGenerateTerminateStateProgram 100313a8 f   pds.obj
 0001:00030450       PDSPatchTerminateStateProgram 10031450 f   pds.obj
 0001:0003045c       WriteEndOfPassUSSECode     1003145c f   pixevent.obj
 0001:00030474       WriteEndOfRenderUSSECode   10031474 f   pixevent.obj
 0001:000304a4       WriteEndOfTileUSSECode     100314a4 f   pixevent.obj
 0001:00030dfc       PVRCombineBlendCodeWithShader 10031dfc f   combiner.obj
 0001:00031044       UCH_CodeHeapCreate         10032044 f   eurasiaconcmn:codeheap.obj
 0001:0003111c       UCH_CodeHeapDestroy        1003211c f   eurasiaconcmn:codeheap.obj
 0001:00031250       UCH_CodeHeapFreeFunc       10032250 f   eurasiaconcmn:codeheap.obj
 0001:000312a4       UCH_CodeHeapAllocateFunc   100322a4 f   eurasiaconcmn:codeheap.obj
 0001:00031794       CBUF_GetBufferSpace        10032794 f   eurasiaconcmn:buffers.obj
 0001:000319d4       CBUF_UpdateBufferPos       100329d4 f   eurasiaconcmn:buffers.obj
 0001:00031a10       CBUF_GetBufferDeviceAddress 10032a10 f   eurasiaconcmn:buffers.obj
 0001:00031a34       CBUF_UpdateBufferCommittedPrimOffsets 10032a34 f   eurasiaconcmn:buffers.obj
 0001:00031abc       CBUF_UpdateBufferCommittedHWOffsets 10032abc f   eurasiaconcmn:buffers.obj
 0001:00031b00       CBUF_UpdateTACtrlKickBase  10032b00 f   eurasiaconcmn:buffers.obj
 0001:00031b50       CBUF_CreateBuffer          10032b50 f   eurasiaconcmn:buffers.obj
 0001:00031c90       CBUF_DestroyBuffer         10032c90 f   eurasiaconcmn:buffers.obj
 0001:00031cac       FRM_Initialize             10032cac f   eurasiaconcmn:frameresource.obj
 0001:00031e7c       FRM_Attach                 10032e7c f   eurasiaconcmn:frameresource.obj
 0001:00031f88       FRM_IsResourceNeeded       10032f88 f   eurasiaconcmn:frameresource.obj
 0001:00032074       FRM_WaitForAllResources    10033074 f   eurasiaconcmn:frameresource.obj
 0001:000320fc       FRM_GhostResource          100330fc f   eurasiaconcmn:frameresource.obj
 0001:0003220c       FRM_RemoveResourceFromAllLists 1003320c f   eurasiaconcmn:frameresource.obj
 0001:000322e4       FRM_RemoveSurfaceReferences 100332e4 f   eurasiaconcmn:frameresource.obj
 0001:00032324       FRM_Destroy                10033324 f   eurasiaconcmn:frameresource.obj
 0001:0003248c       FRM_ReclaimUnneededResources 1003348c f   eurasiaconcmn:frameresource.obj
 0001:0003249c       FRM_DestroyUnneededGhosts  1003349c f   eurasiaconcmn:frameresource.obj
 0001:00033004       DeTwiddleAddress16bpp      10034004 f   eurasiaconcmn:twiddle.obj
 0001:0003317c       ReadBackTwiddle16bpp       1003417c f   eurasiaconcmn:twiddle.obj
 0001:00033d4c       DeTwiddleAddress32bpp      10034d4c f   eurasiaconcmn:twiddle.obj
 0001:00033ec0       ReadBackTwiddle32bpp       10034ec0 f   eurasiaconcmn:twiddle.obj
 0001:00033ff8       ReadBackTwiddle8bpp        10034ff8 f   eurasiaconcmn:twiddle.obj
 0001:000340dc       ReadBackTwiddleETC1        100350dc f   eurasiaconcmn:twiddle.obj
 0001:00034270       DeTwiddleAddress8bpp       10035270 f   eurasiaconcmn:twiddle.obj
 0001:000343d0       DeTwiddleAddressETC1       100353d0 f   eurasiaconcmn:twiddle.obj
 0001:0003454c       PVRUniPatchCreateContext   1003554c f   usp:usp.obj
 0001:000345ac       PVRUniPatchCreateShader    100355ac f   usp:usp.obj
 0001:000345b0       PVRUniPatchCreatePCShader  100355b0 f   usp:usp.obj
 0001:000345b4       PVRUniPatchSetTextureFormat 100355b4 f   usp:usp.obj
 0001:00034610       PVRUniPatchSetOutputLocation 10035610 f   usp:usp.obj
 0001:00034618       PVRUniPatchFinaliseShader  10035618 f   usp:usp.obj
 0001:00034744       PVRUniPatchDestroyHWShader 10035744 f   usp:usp.obj
 0001:00034760       PVRUniPatchDestroyShader   10035760 f   usp:usp.obj
 0001:00034764       PVRUniPatchDestroyPCShader 10035764 f   usp:usp.obj
 0001:0003477c       PVRUniPatchDestroyContext  1003577c f   usp:usp.obj
 0001:00034c04       USPShaderAddResultRef      10035c04 f   usp:uspshader.obj
 0001:00034c34       USPShaderRemoveResultRef   10035c34 f   usp:uspshader.obj
 0001:00037918       USPShaderDestroy           10038918 f   usp:uspshader.obj
 0001:00037ab0       PCShaderCreate             10038ab0 f   usp:uspshader.obj
 0001:00037c08       USPShaderCreate            10038c08 f   usp:uspshader.obj
 0001:00037ef0       HandleUSPSampleTextureFormat 10038ef0 f   usp:finalise.obj
 0001:000380cc       ResetShader                100390cc f   usp:finalise.obj
 0001:000381ac       FinaliseSampleAndResultLocations 100391ac f   usp:finalise.obj
 0001:00038354       FinaliseRegCounts          10039354 f   usp:finalise.obj
 0001:00038424       FinaliseSamples            10039424 f   usp:finalise.obj
 0001:00038498       FinaliseResults            10039498 f   usp:finalise.obj
 0001:000387f0       FinaliseShaderPreamble     100397f0 f   usp:finalise.obj
 0001:0003887c       FinaliseInstructions       1003987c f   usp:finalise.obj
 0001:000388bc       FinaliseBranches           100398bc f   usp:finalise.obj
 0001:00038918       CreateHWShader             10039918 f   usp:finalise.obj
 0001:00039450       USPInstBlockReset          1003a450 f   usp:usp_instblock.obj
 0001:0003973c       USPInstBlockInsertHWInst   1003a73c f   usp:usp_instblock.obj
 0001:000398c0       USPInstBlockAddPCInst      1003a8c0 f   usp:usp_instblock.obj
 0001:00039a78       USPInstBlockRemoveInst     1003aa78 f   usp:usp_instblock.obj
 0001:0003a104       USPInstBlockFinaliseInsts  1003b104 f   usp:usp_instblock.obj
 0001:0003a15c       USPInstBlockCreate         1003b15c f   usp:usp_instblock.obj
 0001:0003a33c       USPInstBlockDestroy        1003b33c f   usp:usp_instblock.obj
 0001:0003a3b8       HWInstGetOpcode            1003b3b8 f   usp:hwinst.obj
 0001:0003ad10       HWInstGetOperandsUsed      1003bd10 f   usp:hwinst.obj
 0001:0003b004       HWInstCanUseExtSrc0Banks   1003c004 f   usp:hwinst.obj
 0001:0003b044       HWInstIsMOEControlInst     1003c044 f   usp:hwinst.obj
 0001:0003b060       HWInstUpdateMOEState       1003c060 f   usp:hwinst.obj
 0001:0003b174       HWInstGetPerOperandFmtCtl  1003c174 f   usp:hwinst.obj
 0001:0003b3dc       HWInstEncodeDestBankAndNum 1003c3dc f   usp:hwinst.obj
 0001:0003b64c       HWInstDecodeDestBankAndNum 1003c64c f   usp:hwinst.obj
 0001:0003b844       HWInstEncodeSrc0BankAndNum 1003c844 f   usp:hwinst.obj
 0001:0003ba1c       HWInstDecodeSrc0BankAndNum 1003ca1c f   usp:hwinst.obj
 0001:0003bb48       HWInstEncodeSrc1BankAndNum 1003cb48 f   usp:hwinst.obj
 0001:0003bd1c       HWInstDecodeSrc1BankAndNum 1003cd1c f   usp:hwinst.obj
 0001:0003beac       HWInstEncodeSrc2BankAndNum 1003ceac f   usp:hwinst.obj
 0001:0003c08c       HWInstDecodeSrc2BankAndNum 1003d08c f   usp:hwinst.obj
 0001:0003c21c       HWInstDecodeOperandBankAndNum 1003d21c f   usp:hwinst.obj
 0001:0003c2dc       HWInstEncodeANDInst        1003d2dc f   usp:hwinst.obj
 0001:0003c45c       HWInstEncodeMOVInst        1003d45c f   usp:hwinst.obj
 0001:0003c4f4       HWInstDecodeMOVInstTestDataType 1003d4f4 f   usp:hwinst.obj
 0001:0003c568       HWInstDecodeRepeat         1003d568 f   usp:hwinst.obj
 0001:0003c6e8       HWInstEncodeSMLSIInst      1003d6e8 f   usp:hwinst.obj
 0001:0003c84c       HWInstEncodeSMBOInst       1003d84c f   usp:hwinst.obj
 0001:0003c8e4       HWInstEncodeSETFCInst      1003d8e4 f   usp:hwinst.obj
 0001:0003c918       HWInstSetBranchOffset      1003d918 f   usp:hwinst.obj
 0001:0003c95c       HWInstSupportsNoSched      1003d95c f   usp:hwinst.obj
 0001:0003c9ac       HWInstSetNoSched           1003d9ac f   usp:hwinst.obj
 0001:0003ca08       HWInstEncodeNOPInst        1003da08 f   usp:hwinst.obj
 0001:0003ca20       HWInstNeedsSyncStartBefore 1003da20 f   usp:hwinst.obj
 0001:0003ca84       HWInstSupportsSyncStart    1003da84 f   usp:hwinst.obj
 0001:0003cacc       HWInstGetSyncStart         1003dacc f   usp:hwinst.obj
 0001:0003cb00       HWInstSetSyncStart         1003db00 f   usp:hwinst.obj
 0001:0003cb38       HWInstSupportsSyncEnd      1003db38 f   usp:hwinst.obj
 0001:0003cb54       HWInstGetSyncEnd           1003db54 f   usp:hwinst.obj
 0001:0003cb70       HWInstForcesDeschedule     1003db70 f   usp:hwinst.obj
 0001:0003cbec       HWInstIsIllegalInstPair    1003dbec f   usp:hwinst.obj
 0001:0003cc68       HWInstSupportsEnd          1003dc68 f   usp:hwinst.obj
 0001:0003ccc0       HWInstSupportsWriteMask    1003dcc0 f   usp:hwinst.obj
 0001:0003ccd4       HWInstDecodeSOPWMInstWriteMask 1003dcd4 f   usp:hwinst.obj
 0001:0003cd20       HWInstDecodeWriteMask      1003dd20 f   usp:hwinst.obj
 0001:0003cd68       HWInstEncodePCKUNPCKInstWriteMask 1003dd68 f   usp:hwinst.obj
 0001:0003ce3c       HWInstEncodeSOPWMInstWriteMask 1003de3c f   usp:hwinst.obj
 0001:0003ceac       HWInstDecodeSMPInstDRCNum  1003deac f   usp:hwinst.obj
 0001:0003ceb8       HWInstEncodeWDFInst        1003deb8 f   usp:hwinst.obj
 0001:0003cee4       HWInstEncodeSOPWMInst      1003dee4 f   usp:hwinst.obj
 0001:0003cfdc       HWInstEncodeSOP2Inst       1003dfdc f   usp:hwinst.obj
 0001:0003d0f8       HWInstDecodeSMPInstCoordFmt 1003e0f8 f   usp:hwinst.obj
 0001:0003d100       HWInstDecodeSMPInstCoordDim 1003e100 f   usp:hwinst.obj
 0001:0003d138       HWInstDecodePCKUNPCKInstSrcFormat 1003e138 f   usp:hwinst.obj
 0001:0003d1a8       HWInstEncodeLDInstFetchCount 1003e1a8 f   usp:hwinst.obj
 0001:0003d1cc       HWInstEncodeLDInst         1003e1cc f   usp:hwinst.obj
 0001:0003d284       HWInstEncodeFIRHInst       1003e284 f   usp:hwinst.obj
 0001:0003d384       HWInstEncodeSMPInstCoordDim 1003e384 f   usp:hwinst.obj
 0001:0003d3d0       HWInstEncodePCKUNPCKInst   1003e3d0 f   usp:hwinst.obj
 0001:0004174c       USPSampleDataAdd           1004274c f   usp:usp_sample.obj
 0001:00041778       USPSampleReset             10042778 f   usp:usp_sample.obj
 0001:00041b30       USPSampleGenerateCode      10042b30 f   usp:usp_sample.obj
 0001:00041c68       USPSampleCreate            10042c68 f   usp:usp_sample.obj
 0001:00041d0c       USPSampleDestroy           10042d0c f   usp:usp_sample.obj
 0001:0004277c       DecideChunksSampling       1004377c f   usp:usp_sample.obj
 0001:000433f8       DecideFinalTextureFormats  100443f8 f   usp:usp_sample.obj
 0001:000434e8       USPInputDataGetPreSampledData 100444e8 f   usp:usp_inputdata.obj
 0001:00043554       USPInputDataGetTexStateData 10044554 f   usp:usp_inputdata.obj
 0001:00043598       USPInputDataCalcPARegUse   10044598 f   usp:usp_inputdata.obj
 0001:00043610       USPInputDataAddTexStateData 10044610 f   usp:usp_inputdata.obj
 0001:000437e8       USPInputDataFixUnusedPreSampledData 100447e8 f   usp:usp_inputdata.obj
 0001:00043830       USPInputDataAddPreSampledData 10044830 f   usp:usp_inputdata.obj
 0001:000439e4       USPInputDataAddIteratedData 100449e4 f   usp:usp_inputdata.obj
 0001:00043b44       USPInputDataGetIteratedDataForNonDepSample 10044b44 f   usp:usp_inputdata.obj
 0001:00043bd4       USPInputDataAddPCInputData 10044bd4 f   usp:usp_inputdata.obj
 0001:00043eec       USPInputDataCreate         10044eec f   usp:usp_inputdata.obj
 0001:00043f1c       USPInputDataCreateIteratedDataList 10044f1c f   usp:usp_inputdata.obj
 0001:00043f64       USPInputDataCreatePreSampledDataList 10044f64 f   usp:usp_inputdata.obj
 0001:00043fb8       USPInputDataCreateTexStateDataList 10044fb8 f   usp:usp_inputdata.obj
 0001:00044008       USPInputDataDestroy        10045008 f   usp:usp_inputdata.obj
 0001:00044064       USPInputDataReset          10045064 f   usp:usp_inputdata.obj
 0001:0004408c       USPResultRefSetup          1004508c f   usp:usp_resultref.obj
 0001:000440bc       USPResultRefCreate         100450bc f   usp:usp_resultref.obj
 0001:00044108       USPResultRefSetInst        10045108 f   usp:usp_resultref.obj
 0001:00044200       USPResultRefDestroy        10045200 f   usp:usp_resultref.obj
 0001:00044220       USPResultRefReset          10045220 f   usp:usp_resultref.obj
 0001:00044240       USPResultRefSupportsRegLocation 10045240 f   usp:usp_resultref.obj
 0001:000443a8       USPResultRefChangeRegLocation 100453a8 f   usp:usp_resultref.obj
 0001:000445e8       PVRSRVPollForValue         100455e8 f   srvclum:SRVCLUM.dll
 0001:000445f8       PVRSRVFreeDeviceMem        100455f8 f   srvclum:SRVCLUM.dll
 0001:00044608       PVRSRVAllocDeviceMem       10045608 f   srvclum:SRVCLUM.dll
 0001:00044618       PVRSRVUnlockMutex          10045618 f   srvclum:SRVCLUM.dll
 0001:00044628       PVRSRVLockMutex            10045628 f   srvclum:SRVCLUM.dll
 0001:00044638       PVRSRVDestroyMutex         10045638 f   srvclum:SRVCLUM.dll
 0001:00044648       PVRSRVCreateMutex          10045648 f   srvclum:SRVCLUM.dll
 0001:00044658       SGXQueueTransfer           10045658 f   srvclum:SRVCLUM.dll
 0001:00044668       PVRSRVFreeAppHintState     10045668 f   srvclum:SRVCLUM.dll
 0001:00044678       PVRSRVGetAppHint           10045678 f   srvclum:SRVCLUM.dll
 0001:00044688       PVRSRVCreateAppHintState   10045688 f   srvclum:SRVCLUM.dll
 0001:00044698       PVRSRVEventObjectWait      10045698 f   srvclum:SRVCLUM.dll
 0001:000446a8       SGXKickTA                  100456a8 f   srvclum:SRVCLUM.dll
 0001:000446b8       PVRSRVGetLibFuncAddr       100456b8 f   srvclum:SRVCLUM.dll
 0001:000446c8       PVRSRVLoadLibrary          100456c8 f   srvclum:SRVCLUM.dll
 0001:000446d8       PVRSRVUnloadLibrary        100456d8 f   srvclum:SRVCLUM.dll
 0001:000446e8       PVRSRVEnumerateDeviceClass 100456e8 f   srvclum:SRVCLUM.dll
 0001:000446f8       PVRSRVCloseBCDevice        100456f8 f   srvclum:SRVCLUM.dll
 0001:00044708       PVRSRVUnmapDeviceClassMemory 10045708 f   srvclum:SRVCLUM.dll
 0001:00044718       PVRSRVMapDeviceClassMemory 10045718 f   srvclum:SRVCLUM.dll
 0001:00044728       PVRSRVGetBCBuffer          10045728 f   srvclum:SRVCLUM.dll
 0001:00044738       PVRSRVGetBCBufferInfo      10045738 f   srvclum:SRVCLUM.dll
 0001:00044748       PVRSRVOpenBCDevice         10045748 f   srvclum:SRVCLUM.dll
 0001:00044758       PVRSRVFreeUserModeMem      10045758 f   srvclum:SRVCLUM.dll
 0001:00044768       PVRSRVCallocUserModeMem    10045768 f   srvclum:SRVCLUM.dll
 0001:00044778       PVRSRVMemSet               10045778 f   srvclum:SRVCLUM.dll
 0001:00044788       PVRSRVAllocUserModeMem     10045788 f   srvclum:SRVCLUM.dll
 0001:00044798       PVRSRVReallocUserModeMem   10045798 f   srvclum:SRVCLUM.dll
 0001:000447a8       KEGLGetDrawableParameters  100457a8 f   libimgegl:libIMGEGL.dll
 0001:000447b8       KEGLDestroyRenderSurface   100457b8 f   libimgegl:libIMGEGL.dll
 0001:000447c8       KEGLUnbindImage            100457c8 f   libimgegl:libIMGEGL.dll
 0001:000447d8       KEGLCreateRenderSurface    100457d8 f   libimgegl:libIMGEGL.dll
 0001:000447e8       KEGLResizeRenderSurface    100457e8 f   libimgegl:libIMGEGL.dll
 0001:000447f8       KEGLBindImage              100457f8 f   libimgegl:libIMGEGL.dll
 0001:00044808       KEGLGetImageSource         10045808 f   libimgegl:libIMGEGL.dll
 0001:00044818       TlsCall                    10045818 f   coredll:COREDLL.dll
 0001:00044828       TlsGetValue                10045828 f   coredll:COREDLL.dll
 0001:00044838       TlsSetValue                10045838 f   coredll:COREDLL.dll
 0001:00044848       DllMain                    10045848 f   corelib0:dllmain.obj
 0001:00044964       _DllMainCRTStartup         10045964 f   corelib0:pegdmain.obj
 0001:00044994       __GSHandlerCheckCommon     10045994 f   corelib0:gshandler.obj
 0001:000449d0       __GSHandlerCheck           100459d0 f   corelib0:gshandler.obj
 0001:000449f4       __security_init_cookie     100459f4 f   corelib0:seccinit.obj
 0001:00044a50       __security_check_cookie    10045a50 f   corelib0:armsecgs.obj
 0001:00044a64       __gsfailure                10045a64 f   corelib0:armsecgs.obj
 0001:00044b70       _cexit                     10045b70 f   corelib0:cexit.obj
 0001:00044b8c       _initterm                  10045b8c f   corelib0:crt0dat.obj
 0001:00044bc0       _cinit                     10045bc0 f   corelib0:crt0dat.obj
 0001:00044bf4       memset                     10045bf4 f   corelib1:COREDLL.dll
 0001:00044c04       free                       10045c04 f   corelib1:COREDLL.dll
 0001:00044c14       realloc                    10045c14 f   corelib1:COREDLL.dll
 0001:00044c24       calloc                     10045c24 f   corelib1:COREDLL.dll
 0001:00044c34       memcpy                     10045c34 f   corelib1:COREDLL.dll
 0001:00044c44       malloc                     10045c44 f   corelib1:COREDLL.dll
 0001:00044c54       strcmp                     10045c54 f   corelib1:COREDLL.dll
 0001:00044c64       strlen                     10045c64 f   corelib1:COREDLL.dll
 0001:00044c74       strncpy                    10045c74 f   corelib1:COREDLL.dll
 0001:00044c84       strcat                     10045c84 f   corelib1:COREDLL.dll
 0001:00044c94       strcpy                     10045c94 f   corelib1:COREDLL.dll
 0001:00044ca4       strncmp                    10045ca4 f   corelib1:COREDLL.dll
 0001:00044cb4       sprintf                    10045cb4 f   corelib1:COREDLL.dll
 0001:00044cc4       atoi                       10045cc4 f   corelib1:COREDLL.dll
 0001:00044cd4       memcmp                     10045cd4 f   corelib1:COREDLL.dll
 0001:00044ce4       _XcptFilter                10045ce4 f   corelib1:COREDLL.dll
 0001:00044cf4       __C_specific_handler       10045cf4 f   corelib1:COREDLL.dll
 0001:00044d04       __security_gen_cookie2     10045d04 f   corelib1:COREDLL.dll
 0001:00044d14       __report_gsfailure         10045d14 f   corelib1:COREDLL.dll
 0001:00044d24       DisableThreadLibraryCalls  10045d24 f   coredll:COREDLL.dll
 0001:00044d34       TerminateProcess           10045d34 f   coredll:COREDLL.dll
 0001:00044d6c       __IMPORT_DESCRIPTOR_SRVCLUM 10045d6c     srvclum:SRVCLUM.dll
 0001:00044d80       __IMPORT_DESCRIPTOR_libIMGEGL 10045d80     libimgegl:libIMGEGL.dll
 0001:00044d94       __IMPORT_DESCRIPTOR_COREDLL 10045d94     coredll:COREDLL.dll
 0001:00044da8       __NULL_IMPORT_DESCRIPTOR   10045da8     srvclum:SRVCLUM.dll
 0002:00000000       __imp_memset               10047000     corelib1:COREDLL.dll
 0002:00000004       __imp_DisableThreadLibraryCalls 10047004     coredll:COREDLL.dll
 0002:00000008       __imp___report_gsfailure   10047008     corelib1:COREDLL.dll
 0002:0000000c       __imp___security_gen_cookie2 1004700c     corelib1:COREDLL.dll
 0002:00000010       __imp___C_specific_handler 10047010     corelib1:COREDLL.dll
 0002:00000014       __imp__XcptFilter          10047014     corelib1:COREDLL.dll
 0002:00000018       __imp___divs               10047018     corelib1:COREDLL.dll
 0002:0000001c       __imp_memcmp               1004701c     corelib1:COREDLL.dll
 0002:00000020       __imp_atoi                 10047020     corelib1:COREDLL.dll
 0002:00000024       __imp___les                10047024     corelib1:COREDLL.dll
 0002:00000028       __imp_sprintf              10047028     corelib1:COREDLL.dll
 0002:0000002c       __imp_strncmp              1004702c     corelib1:COREDLL.dll
 0002:00000030       __imp_strcpy               10047030     corelib1:COREDLL.dll
 0002:00000034       __imp_strcat               10047034     corelib1:COREDLL.dll
 0002:00000038       __imp___negs               10047038     corelib1:COREDLL.dll
 0002:0000003c       __imp___stou               1004703c     corelib1:COREDLL.dll
 0002:00000040       __imp___eqs                10047040     corelib1:COREDLL.dll
 0002:00000044       __imp___gts                10047044     corelib1:COREDLL.dll
 0002:00000048       __imp_strncpy              10047048     corelib1:COREDLL.dll
 0002:0000004c       __imp_strlen               1004704c     corelib1:COREDLL.dll
 0002:00000050       __imp___stoi               10047050     corelib1:COREDLL.dll
 0002:00000054       __imp___subs               10047054     corelib1:COREDLL.dll
 0002:00000058       __imp___adds               10047058     corelib1:COREDLL.dll
 0002:0000005c       __imp___ges                1004705c     corelib1:COREDLL.dll
 0002:00000060       __imp___nes                10047060     corelib1:COREDLL.dll
 0002:00000064       __imp___dtos               10047064     corelib1:COREDLL.dll
 0002:00000068       __imp_floor                10047068     corelib1:COREDLL.dll
 0002:0000006c       __imp___muld               1004706c     corelib1:COREDLL.dll
 0002:00000070       __imp___stod               10047070     corelib1:COREDLL.dll
 0002:00000074       __imp_strcmp               10047074     corelib1:COREDLL.dll
 0002:00000078       __imp___rt_udiv            10047078     corelib1:COREDLL.dll
 0002:0000007c       __imp___lts                1004707c     corelib1:COREDLL.dll
 0002:00000080       __imp___itos               10047080     corelib1:COREDLL.dll
 0002:00000084       __imp_malloc               10047084     corelib1:COREDLL.dll
 0002:00000088       __imp_memcpy               10047088     corelib1:COREDLL.dll
 0002:0000008c       __imp_calloc               1004708c     corelib1:COREDLL.dll
 0002:00000090       __imp_TlsCall              10047090     coredll:COREDLL.dll
 0002:00000094       __imp_TlsGetValue          10047094     coredll:COREDLL.dll
 0002:00000098       __imp_TlsSetValue          10047098     coredll:COREDLL.dll
 0002:0000009c       __imp_TerminateProcess     1004709c     coredll:COREDLL.dll
 0002:000000a0       __imp___muls               100470a0     corelib1:COREDLL.dll
 0002:000000a4       __imp___utos               100470a4     corelib1:COREDLL.dll
 0002:000000a8       __imp_free                 100470a8     corelib1:COREDLL.dll
 0002:000000ac       __imp_realloc              100470ac     corelib1:COREDLL.dll
 0002:000000b0       \177COREDLL_NULL_THUNK_DATA 100470b0     coredll:COREDLL.dll
 0002:000000b4       __imp_PVRSRVUnmapDeviceClassMemory 100470b4     srvclum:SRVCLUM.dll
 0002:000000b8       __imp_PVRSRVFreeDeviceMem  100470b8     srvclum:SRVCLUM.dll
 0002:000000bc       __imp_PVRSRVAllocDeviceMem 100470bc     srvclum:SRVCLUM.dll
 0002:000000c0       __imp_PVRSRVUnlockMutex    100470c0     srvclum:SRVCLUM.dll
 0002:000000c4       __imp_PVRSRVLockMutex      100470c4     srvclum:SRVCLUM.dll
 0002:000000c8       __imp_PVRSRVDestroyMutex   100470c8     srvclum:SRVCLUM.dll
 0002:000000cc       __imp_PVRSRVCreateMutex    100470cc     srvclum:SRVCLUM.dll
 0002:000000d0       __imp_SGXQueueTransfer     100470d0     srvclum:SRVCLUM.dll
 0002:000000d4       __imp_PVRSRVReallocUserModeMem 100470d4     srvclum:SRVCLUM.dll
 0002:000000d8       __imp_PVRSRVAllocUserModeMem 100470d8     srvclum:SRVCLUM.dll
 0002:000000dc       __imp_PVRSRVMemSet         100470dc     srvclum:SRVCLUM.dll
 0002:000000e0       __imp_PVRSRVCallocUserModeMem 100470e0     srvclum:SRVCLUM.dll
 0002:000000e4       __imp_PVRSRVFreeUserModeMem 100470e4     srvclum:SRVCLUM.dll
 0002:000000e8       __imp_PVRSRVOpenBCDevice   100470e8     srvclum:SRVCLUM.dll
 0002:000000ec       __imp_PVRSRVGetBCBufferInfo 100470ec     srvclum:SRVCLUM.dll
 0002:000000f0       __imp_PVRSRVGetBCBuffer    100470f0     srvclum:SRVCLUM.dll
 0002:000000f4       __imp_PVRSRVMapDeviceClassMemory 100470f4     srvclum:SRVCLUM.dll
 0002:000000f8       __imp_PVRSRVPollForValue   100470f8     srvclum:SRVCLUM.dll
 0002:000000fc       __imp_PVRSRVCloseBCDevice  100470fc     srvclum:SRVCLUM.dll
 0002:00000100       __imp_PVRSRVEnumerateDeviceClass 10047100     srvclum:SRVCLUM.dll
 0002:00000104       __imp_PVRSRVUnloadLibrary  10047104     srvclum:SRVCLUM.dll
 0002:00000108       __imp_PVRSRVLoadLibrary    10047108     srvclum:SRVCLUM.dll
 0002:0000010c       __imp_PVRSRVGetLibFuncAddr 1004710c     srvclum:SRVCLUM.dll
 0002:00000110       __imp_SGXKickTA            10047110     srvclum:SRVCLUM.dll
 0002:00000114       __imp_PVRSRVEventObjectWait 10047114     srvclum:SRVCLUM.dll
 0002:00000118       __imp_PVRSRVCreateAppHintState 10047118     srvclum:SRVCLUM.dll
 0002:0000011c       __imp_PVRSRVGetAppHint     1004711c     srvclum:SRVCLUM.dll
 0002:00000120       __imp_PVRSRVFreeAppHintState 10047120     srvclum:SRVCLUM.dll
 0002:00000124       \177SRVCLUM_NULL_THUNK_DATA 10047124     srvclum:SRVCLUM.dll
 0002:00000128       __imp_KEGLDestroyRenderSurface 10047128     libimgegl:libIMGEGL.dll
 0002:0000012c       __imp_KEGLUnbindImage      1004712c     libimgegl:libIMGEGL.dll
 0002:00000130       __imp_KEGLCreateRenderSurface 10047130     libimgegl:libIMGEGL.dll
 0002:00000134       __imp_KEGLResizeRenderSurface 10047134     libimgegl:libIMGEGL.dll
 0002:00000138       __imp_KEGLBindImage        10047138     libimgegl:libIMGEGL.dll
 0002:0000013c       __imp_KEGLGetImageSource   1004713c     libimgegl:libIMGEGL.dll
 0002:00000140       __imp_KEGLGetDrawableParameters 10047140     libimgegl:libIMGEGL.dll
 0002:00000144       \177libIMGEGL_NULL_THUNK_DATA 10047144     libimgegl:libIMGEGL.dll
 0002:0000014c       __security_cookie          1004714c     corelib0:seccinit.obj
 0002:00000150       __security_cookie_complement 10047150     corelib0:seccinit.obj
 0002:00000154       _exitflag                  10047154     corelib0:cexit.obj
 0002:00000158       __onexitend                10047158     <common>
 0002:0000015c       __onexitbegin              1004715c     <common>
 0002:00000160       _pRawDllMain               10047160     <common>

 entry point at        0001:00044964

 Static symbols

 0001:00008024       SetupVerticesForAccum      10009024 f   accum.obj
 0001:00008388       SetupVerticesAndShaderForAccum 10009388 f   accum.obj
 0001:00008a4c       SGXBS_ComputeHash          10009a4c f   binshader.obj
 0001:00008b24       SGXBS_Calloc               10009b24 f   binshader.obj
 0001:00008bac       ReadString                 10009bac f   binshader.obj
 0001:00008c48       ReadU16                    10009c48 f   binshader.obj
 0001:00008c98       ReadU32                    10009c98 f   binshader.obj
 0001:00008cf0       UnpackSymbolBindings       10009cf0 f   binshader.obj
 0001:00008e9c       UnpackSharedShaderState    10009e9c f   binshader.obj
 0001:00009104       UnpackRevision             1000a104 f   binshader.obj
 0001:00009234       UnpackProgramBinary        1000a234 f   binshader.obj
 0001:00009b40       WaitUntilBufObjNotUsed     1000ab40 f   bufobj.obj
 0001:00009bfc       DisposeBufObject           1000abfc f   bufobj.obj
 0001:0000a440       SetupVerticesForClear      1000b440 f   clear.obj
 0001:0000a790       SetupVerticesAndShaderForClear 1000b790 f   clear.obj
 0001:0000a9e8       SetupFragmentShaderForClear 1000b9e8 f   clear.obj
 0001:0000af98       WriteDirect16Indices       1000bf98 f   drawvarray.obj
 0001:0000b0c0       WriteLineStripOrLoop16Indices 1000c0c0 f   drawvarray.obj
 0001:0000b21c       WriteDirect32Indices       1000c21c f   drawvarray.obj
 0001:0000b348       WriteLineStripOrLoop32Indices 1000c348 f   drawvarray.obj
 0001:0000b464       GetNumIndices              1000c464 f   drawvarray.obj
 0001:0000b500       SetupStreamPointers        1000c500 f   drawvarray.obj
 0001:0000b5e8       CopyVArrayData             1000c5e8 f   drawvarray.obj
 0001:0000b6bc       CopyVArrayDataDeindex      1000c6bc f   drawvarray.obj
 0001:0000b8a0       GetVertexIndexBufferSpace  1000c8a0 f   drawvarray.obj
 0001:0000b990       CreateSequentialStaticIndices 1000c990 f   drawvarray.obj
 0001:0000ba34       CreateLineStripStaticIndices 1000ca34 f   drawvarray.obj
 0001:0000badc       GetVArrayBatchRewindCount  1000cadc f   drawvarray.obj
 0001:0000bb54       DrawVertexArray            1000cb54 f   drawvarray.obj
 0001:0000bca0       DrawArraysBatchedStaticIndices 1000cca0 f   drawvarray.obj
 0001:0000bd60       DrawArraysAutoIndices      1000cd60 f   drawvarray.obj
 0001:0000be9c       DrawElementsDeindex        1000ce9c f   drawvarray.obj
 0001:0000bf28       DrawElementsIndexBO        1000cf28 f   drawvarray.obj
 0001:0000c088       DrawBatchOnVBuffer         1000d088 f   drawvarray.obj
 0001:0000c63c       PickDrawArraysProc         1000d63c f   drawvarray.obj
 0001:0000c764       PickDrawElementsProc       1000d764 f   drawvarray.obj
 0001:0000c8d4       DetermineMinAndMaxIndices  1000d8d4 f   drawvarray.obj
 0001:0000c9c0       TransformIndicesTo16Bits   1000d9c0 f   drawvarray.obj
 0001:0000ca54       AttachUsedTexturesToCurrentSurface 1000da54 f   drawvarray.obj
 0001:0000caf4       AttachAllUsedResourcesToCurrentSurface 1000daf4 f   drawvarray.obj
 0001:0000cb44       AttachAllUsedVBOToCurrentKick 1000db44 f   drawvarray.obj
 0001:0000d1c4       MultiDrawArraysAutoIndices 1000e1c4 f   drawvarray.obj
 0001:0000d3a4       MultiDrawBatchOnVBuffer    1000e3a4 f   drawvarray.obj
 0001:0000da4c       MultiDrawVertexArray       1000ea4c f   drawvarray.obj
 0001:0000dc80       MultiDrawElementsDeindex   1000ec80 f   drawvarray.obj
 0001:0000de10       MultiDrawElementsIndexBO   1000ee10 f   drawvarray.obj
 0001:0000dfac       PickMultiDrawElementsProc  1000efac f   drawvarray.obj
 0001:0000e940       FreeContextSharedState     1000f940 f   eglglue.obj
 0001:0000eac4       CreateSharedState          1000fac4 f   eglglue.obj
 0001:0000ecd4       InitContext                1000fcd4 f   eglglue.obj
 0001:0000f104       DeInitContext              10010104 f   eglglue.obj
 0001:0000f1b0       GLES2CreateGC              100101b0 f   eglglue.obj
 0001:0000f228       GLES2DestroyGC             10010228 f   eglglue.obj
 0001:0000f258       GLES2MakeCurrentGC         10010258 f   eglglue.obj
 0001:0000f3b8       GLES2MakeUnCurrentGC       100103b8 f   eglglue.obj
 0001:0000f414       GLES2FlushBuffersGC        10010414 f   eglglue.obj
 0001:0000f488       GLES2MarkRenderSurfaceAsInvalid 10010488 f   eglglue.obj
 0001:0000f4e0       GLES2GetProcAddress        100104e0 f   eglglue.obj
 0001:0000f750       FreeFrameBuffer            10010750 f   fbo.obj
 0001:0000f874       DisposeFrameBufferObject   10010874 f   fbo.obj
 0001:0000f878       DisposeRenderBuffer        10010878 f   fbo.obj
 0001:0000fcd0       ComputeFrameBufferCompleteness 10010cd0 f   fbo.obj
 0001:0001049c       NotifyFrameBuffer          1001149c f   fbo.obj
 0001:00011718       ConvertResult              10012718 f   get.obj
 0001:00011c1c       IsEnabled                  10012c1c f   get.obj
 0001:00011d34       GetBlendFactor             10012d34 f   get.obj
 0001:00011e08       GetStencilOp               10012e08 f   get.obj
 0001:00011ea0       DoGet                      10012ea0 f   get.obj
 0001:000135c8       GetTexParameter            100145c8 f   get.obj
 0001:000140ac       HardwareMipTextureTransfer 100150ac f   makemips.obj
 0001:00014360       HardwareMipGen             10015360 f   makemips.obj
 0001:000145d4       MakeMapLevel16bpp          100155d4 f   makemips.obj
 0001:000148f8       MakeMapLevel32bpp          100158f8 f   makemips.obj
 0001:00014ad0       SetupMipmapTextureControlWords 10015ad0 f   makemips.obj
 0001:00014d1c       HardwareMakeTextureMipmapLevels 10015d1c f   makemips.obj
 0001:00015a68       FloatToHWByte              10016a68 f   misc.obj
 0001:00016bd8       CheckReadPixelArgs         10017bd8 f   pixelop.obj
 0001:000174e0       CalcRegionClip             100184e0 f   scissor.obj
 0001:000175a0       SetupVerticesForDrawmask   100185a0 f   scissor.obj
 0001:0001784c       SetupVerticesAndShaderForDrawmask 1001884c f   scissor.obj
 0001:00017a98       SendDrawMaskRect           10018a98 f   scissor.obj
 0001:00018170       SetupZLSRegs               10019170 f   sgxif.obj
 0001:000183b4       GLES2InitRegs              100193b4 f   sgxif.obj
 0001:0001847c       StartFrame                 1001947c f   sgxif.obj
 0001:000188bc       DoKickTA                   100198bc f   sgxif.obj
 0001:0001914c       CopySymbolBindings         1001a14c f   shader.obj
 0001:00019370       CreateSharedShaderState    1001a370 f   shader.obj
 0001:00019b98       LoadCompilerModule         1001ab98 f   shader.obj
 0001:00019cc4       SetPrecision               1001acc4 f   shader.obj
 0001:00019e38       InitializeGLSLCompiler     1001ae38 f   shader.obj
 0001:00019fe0       AssignAttributeLocations   1001afe0 f   shader.obj
 0001:0001a280       AttributeCompileMask       1001b280 f   shader.obj
 0001:0001a33c       SetupProgramOutputSelects  1001b33c f   shader.obj
 0001:0001a428       CountAttribUniformVaryings 1001b428 f   shader.obj
 0001:0001a4e4       AddNewUniforms             1001b4e4 f   shader.obj
 0001:0001a714       AddFragmentProgramUniforms 1001b714 f   shader.obj
 0001:0001a92c       AppendMessageToProgramInfoLog 1001b92c f   shader.obj
 0001:0001a9b8       LinkVertexFragmentPrograms 1001b9b8 f   shader.obj
 0001:0001b088       UseProgram                 1001c088 f   shader.obj
 0001:0001b8cc       SharedShaderStateDelRef    1001c8cc f   shader.obj
 0001:0001b9e4       FreeListOfVertexUSEVariants 1001c9e4 f   shader.obj
 0001:0001ba6c       FreeListOfFragmentUSEVariants 1001ca6c f   shader.obj
 0001:0001bbc0       ResetProgramLinkedState    1001cbc0 f   shader.obj
 0001:0001c4a0       FreeProgram                1001d4a0 f   shader.obj
 0001:0001c5e0       DisposeProgram             1001d5e0 f   shader.obj
 0001:0001d46c       BlendFuncSeparate          1001e46c f   state.obj
 0001:0001dd6c       StencilFunc                1001ed6c f   state.obj
 0001:0001df8c       StencilMask                1001ef8c f   state.obj
 0001:0001e110       StencilOp                  1001f110 f   state.obj
 0001:0001eddc       CopyTexturePVRTC           1001fddc f   tex.obj
 0001:0001ee58       CopyTextureETC1            1001fe58 f   tex.obj
 0001:0001f73c       TexParameterfv             1002073c f   tex.obj
 0001:0001fe78       CheckTexImageArgs          10020e78 f   tex.obj
 0001:0001ff64       CheckTexSubImageArgs       10020f64 f   tex.obj
 0001:000200f0       UpdateEGLImage             100210f0 f   tex.obj
 0001:00022ba4       HardwareTextureTransfer    10023ba4 f   texdata.obj
 0001:00024484       ReadBackMultiChunkData     10025484 f   texdata.obj
 0001:00025184       UnloadInconsistentTexture  10026184 f   texmgmt.obj
 0001:00025cac       FreeTexture                10026cac f   texmgmt.obj
 0001:00025de8       DisposeTexObj              10026de8 f   texmgmt.obj
 0001:00025dec       CreateDummyTextures        10026dec f   texmgmt.obj
 0001:00026da4       SaveUniformDataFloat       10027da4 f   uniform.obj
 0001:00027120       SaveUniformDataInteger     10028120 f   uniform.obj
 0001:000288d0       EncodeTwoSourceBlend       100298d0 f   use.obj
 0001:00028a18       EncodeThreeSourceBlend     10029a18 f   use.obj
 0001:00029020       InitStateCopyUSECodeBlocks 1002a020 f   use.obj
 0001:000291f0       CreateVertexUnpackUSECode  1002a1f0 f   use.obj
 0001:0002985c       SetupUSESecondaryUploadTask 1002a85c f   use.obj
 0001:00029d74       SetupIteratorsAndTextureLookups 1002ad74 f   use.obj
 0001:0002ac58       WritePDSPixelShaderProgram 1002bc58 f   validate.obj
 0001:0002b314       WritePDSVertexShaderProgram 1002c314 f   validate.obj
 0001:0002b9c0       LoadSecondaryAttributes    1002c9c0 f   validate.obj
 0001:0002be04       WritePDSUSEShaderSAProgram 1002ce04 f   validate.obj
 0001:0002c2a0       WriteMTEState              1002d2a0 f   validate.obj
 0001:0002c8d4       SetupAttribStreams         1002d8d4 f   validate.obj
 0001:0002cb04       SetupRenderState           1002db04 f   validate.obj
 0001:0002cf90       WriteVDMControlStream      1002df90 f   validate.obj
 0001:0002d67c       Copy1Byte                  1002e67c f   vertex.obj
 0001:0002d69c       Copy3Bytes                 1002e69c f   vertex.obj
 0001:0002d6d4       Copy1Short                 1002e6d4 f   vertex.obj
 0001:0002d6f4       Copy3Shorts                1002e6f4 f   vertex.obj
 0001:0002d72c       Copy1Long                  1002e72c f   vertex.obj
 0001:0002d74c       Copy2Longs                 1002e74c f   vertex.obj
 0001:0002d77c       Copy3Longs                 1002e77c f   vertex.obj
 0001:0002d7b4       Copy4Longs                 1002e7b4 f   vertex.obj
 0001:0002d7f4       MemCopy1Byte               1002e7f4 f   vertex.obj
 0001:0002d810       MemCopy3Bytes              1002e810 f   vertex.obj
 0001:0002d82c       MemCopy1Short              1002e82c f   vertex.obj
 0001:0002d848       MemCopy3Shorts             1002e848 f   vertex.obj
 0001:0002d868       MemCopy1Long               1002e868 f   vertex.obj
 0001:0002d884       MemCopy2Longs              1002e884 f   vertex.obj
 0001:0002d8a0       MemCopy3Longs              1002e8a0 f   vertex.obj
 0001:0002d8c0       MemCopy4Longs              1002e8c0 f   vertex.obj
 0001:0002d8dc       Copy2Bytes                 1002e8dc f   vertex.obj
 0001:0002d90c       Copy4Bytes                 1002e90c f   vertex.obj
 0001:0002d94c       Copy6Bytes                 1002e94c f   vertex.obj
 0001:0002d988       Copy8Bytes                 1002e988 f   vertex.obj
 0001:0002d9c4       Copy12Bytes                1002e9c4 f   vertex.obj
 0001:0002da00       Copy16Bytes                1002ea00 f   vertex.obj
 0001:0002da3c       Copy2Shorts                1002ea3c f   vertex.obj
 0001:0002da6c       Copy4Shorts                1002ea6c f   vertex.obj
 0001:0002daac       Copy6Shorts                1002eaac f   vertex.obj
 0001:0002dae8       Copy8Shorts                1002eae8 f   vertex.obj
 0001:0002e6dc       InitialiseYUVCoefficients  1002f6dc f   texstream.obj
 0001:0002ec08       CreateTextureStreamState   1002fc08 f   texstream.obj
 0001:0002f4cc       PDSEncodeSimpleMOVS        100304cc f   pds.obj
 0001:0002f5ec       PDSGetNextConstant         100305ec f   pds.obj
 0001:0002f630       PDSGetNumConstants         10030630 f   pds.obj
 0001:00030564       ReplaceArgument            10031564 f   combiner.obj
 0001:00030688       GetSource                  10031688 f   combiner.obj
 0001:00030730       ReplaceArguments           10031730 f   combiner.obj
 0001:000309e4       CombineSOPs                100319e4 f   combiner.obj
 0001:00031188       CodeHeapInsertBlockInFreeList 10032188 f   eurasiaconcmn:codeheap.obj
 0001:000315c4       GetBufferSpaceLeftInBytes  100325c4 f   eurasiaconcmn:buffers.obj
 0001:0003162c       CheckUSSEBufferSpace       1003262c f   eurasiaconcmn:buffers.obj
 0001:00031700       CheckTACtrlBufferSpace     10032700 f   eurasiaconcmn:buffers.obj
 0001:00031dc4       AllocAttachment            10032dc4 f   eurasiaconcmn:frameresource.obj
 0001:00031fe8       WaitUntilResourceIsNotNeeded 10032fe8 f   eurasiaconcmn:frameresource.obj
 0001:00032150       RemoveResourceFromAllLists 10033150 f   eurasiaconcmn:frameresource.obj
 0001:00032238       RemoveSurfaceReferencesInList 10033238 f   eurasiaconcmn:frameresource.obj
 0001:00032398       ReclaimUnneededResourcesInList 10033398 f   eurasiaconcmn:frameresource.obj
 0001:000324ac       InitLookupTable32          100334ac f   eurasiaconcmn:twiddle.obj
 0001:000325f4       Write8x8Pixels16bpp        100335f4 f   eurasiaconcmn:twiddle.obj
 0001:000328c8       TwiddleSmallTexture16bpp   100338c8 f   eurasiaconcmn:twiddle.obj
 0001:00032a4c       Twiddle32x3216bpp          10033a4c f   eurasiaconcmn:twiddle.obj
 0001:00032c34       RecursiveTwid16bpp         10033c34 f   eurasiaconcmn:twiddle.obj
 0001:00032d00       TwiddleRectangularTexture16bpp 10033d00 f   eurasiaconcmn:twiddle.obj
 0001:000330a4       Untwiddle16Bpp             100340a4 f   eurasiaconcmn:twiddle.obj
 0001:000332b4       Write8x8Pixels32bpp        100342b4 f   eurasiaconcmn:twiddle.obj
 0001:000335fc       TwiddleSmallTexture32bpp   100345fc f   eurasiaconcmn:twiddle.obj
 0001:00033780       Twiddle32x3232bpp          10034780 f   eurasiaconcmn:twiddle.obj
 0001:00033958       RecursiveTwid32bpp         10034958 f   eurasiaconcmn:twiddle.obj
 0001:00033a24       TwiddleRectangularTexture32bpp 10034a24 f   eurasiaconcmn:twiddle.obj
 0001:00033dec       Untwiddle32bpp             10034dec f   eurasiaconcmn:twiddle.obj
 0001:000341e8       getUV                      100351e8 f   eurasiaconcmn:twiddle.obj
 0001:00034790       USPProgDescCreate          10035790 f   usp:uspshader.obj
 0001:00034990       USPProgDescDestroy         10035990 f   usp:uspshader.obj
 0001:00034a28       USPShaderAddInstBlock      10035a28 f   usp:uspshader.obj
 0001:00034ae4       USPShaderAddLabel          10035ae4 f   usp:uspshader.obj
 0001:00034c7c       ReadUINT32Straight         10035c7c f   usp:uspshader.obj
 0001:00034cb0       ReadUINT32Swapped          10035cb0 f   usp:uspshader.obj
 0001:00034cdc       ReadUINT16Straight         10035cdc f   usp:uspshader.obj
 0001:00034d00       ReadUINT16Swapped          10035d00 f   usp:uspshader.obj
 0001:00034d1c       WriteUINT32Straight        10035d1c f   usp:uspshader.obj
 0001:00034d58       WriteUINT16Straight        10035d58 f   usp:uspshader.obj
 0001:00034d84       WriteAddSizeUINT32         10035d84 f   usp:uspshader.obj
 0001:00034d94       WriteAddSizeUINT16         10035d94 f   usp:uspshader.obj
 0001:00034da4       USPShaderAddPCInstBlock    10035da4 f   usp:uspshader.obj
 0001:00034ea0       ReadPCHWCodeBlock          10035ea0 f   usp:uspshader.obj
 0001:000351b0       WritePCProgDescBlock       100361b0 f   usp:uspshader.obj
 0001:00035ad4       ReadPCProgDescBlock        10036ad4 f   usp:uspshader.obj
 0001:000364f0       AddNewTextureFormat        100374f0 f   usp:uspshader.obj
 0001:00036634       ReadPCSampleBlock          10037634 f   usp:uspshader.obj
 0001:00036d04       ReadPCBranchBlock          10037d04 f   usp:uspshader.obj
 0001:00036e98       WriteUSPMOEState           10037e98 f   usp:uspshader.obj
 0001:00036f50       WriteUSPSampleBlock        10037f50 f   usp:uspshader.obj
 0001:000373b0       WriteUSPHWCodeBlock        100383b0 f   usp:uspshader.obj
 0001:000374d0       WriteUSPBlocks             100384d0 f   usp:uspshader.obj
 0001:00037818       SetupInputData             10038818 f   usp:uspshader.obj
 0001:0003956c       USPInstDescSetup           1003a56c f   usp:usp_instblock.obj
 0001:000396a8       USPInstBlockInserInst      1003a6a8 f   usp:usp_instblock.obj
 0001:00039b0c       USPInstBlockSetupNoSchedFlag 1003ab0c f   usp:usp_instblock.obj
 0001:00039fc0       USPInstBlockSetupSyncStartFlag 1003afc0 f   usp:usp_instblock.obj
 0001:0003a8a4       HWInstGetOperandsUsedEFO   1003b8a4 f   usp:hwinst.obj
 0001:0003aa18       HWInstGetOperandsUsedPCKUNPCK 1003ba18 f   usp:hwinst.obj
 0001:0003aadc       HWInstGetOperandsUsedSOP2  1003badc f   usp:hwinst.obj
 0001:0003ac44       HWInstGetOperandsUsedSOPWM 1003bc44 f   usp:hwinst.obj
 0001:0003b288       HWInstDecodeIndexedOperandNum 1003c288 f   usp:hwinst.obj
 0001:0003b320       HWInstEncodeIndexedOperandNum 1003c320 f   usp:hwinst.obj
 0001:0003d648       GetTexChanInfo             1003e648 f   usp:usp_sample.obj
 0001:0003dab0       SaveInternalRegs           1003eab0 f   usp:usp_sample.obj
 0001:0003de28       ReStoreInternalRegs        1003ee28 f   usp:usp_sample.obj
 0001:0003e068       SampleTextureData          1003f068 f   usp:usp_sample.obj
 0001:0003e740       ColourSpaceConvertTextureData 1003f740 f   usp:usp_sample.obj
 0001:0003eb84       FindPreSampledTextureData  1003fb84 f   usp:usp_sample.obj
 0001:0003ed94       SetupChanSrcRegs           1003fd94 f   usp:usp_sample.obj
 0001:0003f1e8       SampleInstReadsReg         100401e8 f   usp:usp_sample.obj
 0001:0003f400       UnpackChunksFromTemp       10040400 f   usp:usp_sample.obj
 0001:0003f644       UnpackTextureDataToF32     10040644 f   usp:usp_sample.obj
 0001:0003fc58       UnpackTextureDataToU8C10   10040c58 f   usp:usp_sample.obj
 0001:00040e44       UnpackTextureDataToF16     10041e44 f   usp:usp_sample.obj
 0001:00041668       AddSampleCode              10042668 f   usp:usp_sample.obj
 0001:000417f8       ResetMOEStateBeforeSample  100427f8 f   usp:usp_sample.obj
 0001:00041944       RestoreMOEStateAfterSample 10042944 f   usp:usp_sample.obj
 0001:00041d20       AddSampleToTexChunksSamplesGroup 10042d20 f   usp:usp_sample.obj
 0001:00041eb8       GroupTexChunksSamplesByTexCoords 10042eb8 f   usp:usp_sample.obj
 0001:00042128       DoSelectionsForMinimumPAUsage 10043128 f   usp:usp_sample.obj
 0001:00042338       DoMaxPAAndEntriesUsage     10043338 f   usp:usp_sample.obj
 0001:00042af8       SetDefaultTextureControlWords 10043af8 f   usp:usp_sample.obj
 0001:00042d0c       GenerateUSPTextureFormatInfo 10043d0c f   usp:usp_sample.obj
 0001:0004328c       DecideTextureFormat        1004428c f   usp:usp_sample.obj
 0001:00044868       _DllMainCRTStartupHelper   10045868 f   corelib0:pegdmain.obj
 0001:00044aa8       doexit                     10045aa8 f   corelib0:cexit.obj
